:020000040000FA
:100000000004040000000000041A0000081A0000A8
:100010000C1A0000101A0000141A00000C1B00003B
:100020000C1B00000C1B0000181A00001C1A00001A
:10003000201A0000241A00000C1B0000281A0000DF
:100040002C1A0000301A0000341A0000381A000080
:100050003C1A0000401A0000441A0000481A000030
:100060000C1B00000C1B00004C1A0000501A000072
:10007000541A0000581A00005C1A00000C1B000003
:10008000601A0000641A00000C1B0000681A0000CF
:100090006C1A0000701A0000741A0000781A000030
:1000A0007C1A0000801A0000841A0000881A0000E0
:1000B0000C1B00000C1B00000C1B00008C1A000025
:1000C000901A0000941A0000981A00009C1A000070
:1000D000A01A0000A41A0000A81A0000AC1A000020
:1000E0000C1B00000C1B00000C1B0000B01A0000D1
:1000F000B41A00000C1B00000C1B0000B81A000012
:10010000BC1A00000C1B00000C1B00000C1B0000A4
:100110000C1B00000C1B00000C1B00000C1B000043
:10012000C01A00000C1B00000C1B0000C41A0000C9
:10013000C81A0000CC1A00000C1B00000C1B0000A9
:100140000C1B00000C1B0000D01A00000C1B000050
:100150000C1B00000C1B00000C1B0000D41A00003C
:100160000C1B00000C1B00000C1B0000D81A000028
:10017000DC1A0000E01A0000E41A0000E81A00008F
:10018000EC1A0000F01A0000F41A0000F81A00003F
:10019000FC1A0000001B0000041B0000081B0000EC
:1001A0000C1B00000C1B00000C1B00000C1B0000B3
:1001B0000C1B00000C1B00000C1B00000C1B0000A3
:1001C0000C1B00000C1B00000C1B00000C1B000093
:1001D0000C1B00000C1B00000C1B00000C1B000083
:1001E0000C1B00000C1B00000C1B00000C1B000073
:1001F0000C1B00000C1B00000C1B00000C1B000063
:10020000FFFFFF00FFFFFF00C8040000C80400005C
:10021000C8040000C8040000C8040000C8040000AE
:10022000C8040000C8040000C8040000C80400009E
:10023000C8040000C8040000C8040000C80400008E
:10024000C8040000C8040000C8040000C80400007E
:10025000C8040000C8040000C8040000C80400006E
:10026000C8040000C8040000C8040000C80400005E
:10027000C8040000C8040000C8040000C80400004E
:10028000C8040000C8040000C8040000C80400003E
:10029000C8040000C8040000C8040000C80400002E
:1002A000C8040000C8040000C8040000C80400001E
:1002B000C8040000C8040000C8040000C80400000E
:1002C000C8040000C8040000C8040000C8040000FE
:1002D000C8040000C8040000C8040000C8040000EE
:1002E000C8040000C8040000C8040000C8040000DE
:1002F000C8040000C8040000C8040000C8040000CE
:10030000C8040000C8040000C8040000C8040000BD
:10031000C8040000C8040000C8040000C8040000AD
:10032000C8040000C8040000C8040000C80400009D
:10033000C8040000C8040000C8040000C80400008D
:10034000C8040000C8040000C8040000C80400007D
:10035000C8040000C8040000C8040000C80400006D
:10036000C8040000C8040000C8040000C80400005D
:10037000C8040000C8040000C8040000C80400004D
:10038000C8040000C8040000C8040000C80400003D
:10039000C8040000C8040000C8040000C80400002D
:1003A000C8040000C8040000C8040000C80400001D
:1003B000C8040000C8040000C8040000C80400000D
:1003C000C8040000C8040000C8040000C8040000FD
:1003D000C8040000C8040000C8040000C8040000ED
:1003E000C8040000C8040000C8040000C8040000DD
:1003F000C8040000C8040000C8040000C8040000CD
:100800000FA220000E7F24000E01880000000000CF
:10081000000020000000E000020032000001200083
:1008200020028800140007005B0007000000E000C1
:1008300003003A0080682100010020000200370018
:100840000000200001002000810F70000100320034
:1008500014000700000020000000E0000200320049
:100860000000020000000000DC1402000000000094
:100870000040DA000000FE004440A90040112000C2
:100880000000E0000300320000002000A00188000A
:100890004440A800000006008A1F78008B1F7800E3
:1008A0000000060091018800800478000000EB0041
:1008B0001A003700E284440032A0B4009905BA005F
:1008C000E284440032A0B4009906BA00E2844400F5
:1008D00032A0B4000006EB00476FDE00FD07B20057
:1008E000636CE10003003A00EBFF07000000EB003F
:1008F0000A003700606CE10004003A00005DEB0084
:100900008B05E900FDFF3E00040037006168E1004F
:10091000010032000086EB000B00070019C7BA0087
:100920001905BA000E04E00003003A000A00E000D6
:10093000E0FF3A0000000600FE07B2009E018800BA
:100940008A047800F5FF3700395DBA008B05E900AD
:100950000C003200295DBA008B05E9000800320066
:100960000C00E00003003A00E284440032A0B4002E
:10097000F5FF370019DDBA008B05E900FAFF3A00F0
:100980008904E800E184440032A0B40000000600BD
:100990000040DA000000FE00000005008001780041
:1009A00002003700815978000201E9000200E000EE
:1009B000FCFF3A00000006001201000000020000E7
:1009C0000000000000080000D80400003C00000007
:1009D0000001000001020000000100000902000007
:1009E000290000000101000000C0000032090000E1
:1009F00004000000000200000300000000000000EE
:100A0000092100001101000000010000221D00006A
:100A10000007000005810000034000000001000005
:100A20000705000001030000400000000100000075
:100A30000403000009040000340300004D0000001E
:100A40006900000063000000720000006F000000F9
:100A500063000000680000006900000070000000F2
:100A6000200000005400000065000000630000004A
:100A7000680000006E0000006F0000006C000000C5
:100A80006F000000670000007900000020000000F7
:100A9000490000006E000000630000002E0000000E
:100AA0002603000055000000530000004200000033
:100AB0002000000048000000490000004400000041
:100AC00020000000420000006F0000006F000000E6
:100AD000740000006C0000006F0000006100000066
:100AE00064000000650000007200000006000000C5
:100AF000FF09000001A10000011900000129000008
:100B00004015000000260000FF00000075080000EE
:100B100095400000810000001901000029400000FC
:100B200091000000C0000000EE8400001885000065
:100B30001C850000508500004572000061730000B4
:100B4000696E0000672000004465000076690000BF
:100B5000636500002E2E00002E000000457200008C
:100B60006173000065200000436F00006D7000009D
:100B70006C65000074650000005700007269000099
:100B800074650000204300006F6D0000706C000071
:100B900065740000650A0000507200006573000073
:100BA00073200000526500007365000074000000AF
:100BB000526500007365000074000000754D000070
:100BC0004F470000493200000A4200004F4F00002A
:100BD000544C00004F41000044450000520000000A
:100BE0000080FB008181FB00000140000281410088
:100BF0004311DD0003A020000301410012F0A10019
:100C00000104E00004003A0000004000A180200040
:100C1000823078000300370000004000E1802000AF
:100C20008230780012E0A1006401410012E0A000CF
:100C300000000600214A800080C0B300E78F50000A
:100C40000E003E0001407800818120009140780034
:100C50000104E00004003A0013C0B30082812000C8
:100C60000349780005003700E1CF500003003A0047
:100C700023C0B30082812000034978004194200002
:100C80000081FB00910811007140800080487800CD
:100C9000A1952000D1408800219420009100780087
:100CA000E1806000030032000004E0000C003A0024
:100CB000000006000004E000110032000294200051
:100CC00092017800D140800093587800D14088008C
:100CD0000309E8000040E900F8FF3A0000000600C0
:100CE0000294200092017800D1408000935878004F
:100CF000D14088000309E8000040E900F8FF3A000D
:100D00000000060000C8B30021952000914F10009C
:100D100033003A0001CCB300209420000148780051
:100D20005095200010407800E24F5000090032003A
:100D3000E34F500019003200E14F500026003A0006
:100D4000C04D2800004A880020012000204A880069
:100D500000000600409520001004E0000C003A005E
:100D60001080FB000000400041592800610078001D
:100D7000004A880041942000204190008248780079
:100D80008100E800304090008048780000000600B4
:100D9000209420000048EB00000006004095200051
:100DA00021C0B30090CF100008003E001080FB006F
:100DB000000040006159280061007800004A880066
:100DC0001080FB00204A88000000060020942000CC
:100DD0000048EB0000000600209420000048EB00D3
:100DE000000006000040EB00A1952000804878003C
:100DF0008100E800804878002095200010407800AD
:100E00007F4060000080FB00E10F50000B003200CB
:100E1000E20F50000C0032000000E00028003A0011
:100E2000209420001070A0000348E200240032004B
:100E30000100E9001014A0002100370020942000D8
:100E40001070A0001E003700209420001070A00039
:100E500060952000104078006F406000180032005C
:100E6000609520001004E000070035001040780075
:100E70006F4060000080FB0000004000A180200067
:100E8000E1007800070037006095200010407800EE
:100E90006F4060000080FB0000004000E180200007
:100EA000E10078000040280091006000808F500031
:100EB00003003A0011C0B300A0952000014878005B
:100EC000000820002194200011006000070032007B
:100ED000A0952000004A8800010078001000A000C2
:100EE00021C0B3000080E80001487800000006003F
:100EF000AA24AB0011003200A040800010419000F5
:100F000001C8B300814F51000B003A0071408000CE
:100F10001141900041C8B300814F510006003A00D2
:100F2000C1C0B30011409800A040800090409000E4
:100F30000174A00011409800AA24A9000008200014
:100F40005024880000000600881F78007040800050
:100F5000100478004E44DE00614464000020A200CA
:100F60007040880030408000E80F50000B003A00CD
:100F7000409520001080FB00F007B200B0248800EC
:100F80009604E20003003200000120003040880097
:100F900002003700400020003040880019C8BF0020
:100FA000E14F500021003A00A195200070408000E0
:100FB000110098001FFF070018C8BF00E24F500043
:100FC00008003A0041C0B300704080001140980012
:100FD00070408000904090000174A0001140980083
:100FE000200037000804E00008003A0081C4B30084
:100FF0007040800011409800704080009040900048
:101000000174A000114098001600370081C0B300A1
:101010007040800011409800704080009040900027
:101020000174A000114098000E0037008094200049
:101030001004E0000A003D00514A8000C808DE00AC
:10104000640040001080FB004800DD00008070005C
:101050000100320000000100809420001070A10007
:101060001968EF004F047800000006000468EF00E4
:101070000001EB008200780040072000ED0507002A
:101080008284A90000012000002488000968EF0084
:10109000000006008284A80000012000502488007F
:1010A00010C0B30004E8B7000968EF000001EB00CE
:1010B0008200780050072000DE053700889FBE00C0
:1010C0004095200011C0B30090CF10000E003A00F0
:1010D0000080E900104078007F4060000A003A007C
:1010E000209420001070A0003095200032C0B30082
:1010F000904F110003003A000140780003E8B70068
:10110000010037000368EF00409520001004E00064
:101110009C003A000080E900104078007F406000A9
:10112000E24F500097003A00609520001040780090
:101130006F406000930032006095200010407800FE
:101140006F4060000080FB00E10F50008D003C000C
:10115000000220000608E3008A003A0020942000E4
:101160001070A000609520001004E0000C00350015
:1011700010417800EF4061008180FB0081804000D9
:10118000A280200062847800104078006F406000E8
:101190000080FB0001952000E14478000C0037003E
:1011A0006095200010417800EF4061008180FB00D5
:1011B00081804000E2802000628478001040780046
:1011C0006F4060000080FB00E1942000E144780063
:1011D0000908A30002003A000820A100010037001E
:1011E0000820A000609520001004E00007003500F2
:1011F000104078006F4060000080FB00000040005D
:10120000A18020008830780007003700609520001A
:10121000104078006F4060000080FB00000040003C
:10122000E1802000883078003095200031C0B30084
:1012300090CF10001A003A001800E00013003D00A3
:10124000630040001004E000080035001040780002
:101250006F4060000080FB00019520006141780034
:101260000214A0008270780008003700609520000A
:10127000104078006F4060000080FB00E194200087
:10128000614178000214A0008270780098409000BC
:1012900040C8B30000C07000104498003900370007
:1012A000880078000120A2001100E00008003D0045
:1012B000114090000074A1000064A00090409800CC
:1012C00022002000500020005A05070003003700CC
:1012D000114090000064A000904098000918A300FD
:1012E00002003A001800E0001B003D00609520005D
:1012F0001004E00008003500104078006F406000E6
:101300000080FB0001952000614178000214A100DB
:101310008270780008003700609520001040780047
:101320006F4060000080FB00E19420006141780084
:101330000214A1008270780018409000B043B200FF
:1013400010449800220020008800780050002000FF
:10135000380507000300370018409000B043B20082
:101360001044980060952000104078006F406000A5
:101370000080FB0000004000A14A20000100400066
:101380001014A1004F04BE0000000600881F780062
:10139000209420001070A000AC24EF0008A02000D2
:1013A000020220008000EB00080078007BFD0700AF
:1013B0009424A8000040EB00E194200080487800CD
:1013C0000195200080487800F19420008048780042
:1013D00011952000804878001268EF009424A9003D
:1013E0006800440070408800A8408800B840880029
:1013F000409520001040780008E8B7000004E000A5
:1014000003003A0000012000304088000600370049
:1014100012002000818020000200780005050700EE
:1014200000022000304088004F04780000000600D1
:101430002095200001C6B30010C060003F003A00B4
:10144000309520001080FB008000EB00EB0F500077
:10145000E08F580039003E00006001001C0037009A
:101460001C003700350037001A0037003300370002
:10147000060037000A0037002C0037000A0037004A
:1014800008003700140037002000370020942000A7
:101490001070A0008000200030408800000006008E
:1014A00018FE3700B9FF370080802000004A88000E
:1014B000209420009000780013C0B3000081E80061
:1014C000034978001108B300010878000000060005
:1014D00044FE3700F9FE3700609520001081FB00C4
:1014E0002181200000942000010841000080E800D4
:1014F0009000780013C0B3000081E8000349780031
:101500001108B300010878000000060020942000B4
:101510001070A000609520009080FB0020812000CA
:101520004295200092707800000006000001EB0058
:101530008200780020002000BE04070000000600A2
:101540009EC0A9000080EB00702488005024880011
:10155000AA24EF00AC24EF002000200030258800F2
:10156000A824EF008644A900F00920008024880008
:101570006024880082C4A8008804A80000A020007D
:10158000C800DE00C12488000008EB00301078009D
:101590006000B8002050880031508800405088001A
:1015A0005150880060508800715088008050880039
:1015B00091508800A0508800B1508800C050880029
:1015C000D1508800E0508800F15088009424A80091
:1015D0009624EF0094A4A9009424A9008000200080
:1015E000502488008A64AB00FCFF3A000040EB0006
:1015F0002194200080487800819420000081FB0025
:10160000820878008180E80002F02F0091086100D4
:1016100013C0B30002822000034978001282200028
:10162000034978000268EF000068EF000468EF00EB
:101630000A28EF00E19420008048780001952000FE
:10164000804878001028EF000C28EF00F19420006B
:1016500080487800119520008048780080A0200004
:1016600070408800D0002000502588002095200080
:101670001050880081C0B30000A02000014878000D
:101680000000E80041C0B300014878001074A000D9
:101690000868EF002228EF002428EF000968EF0017
:1016A0000628EF0000000600889FBE008A1F780011
:1016B00000457800814478000984FB000838A300C5
:1016C000030032008040EB000A40780044FD070030
:1016D0000828A3000300320011C0B3000A407800BC
:1016E0003FFD07000A85FB000A054500A04A2000CF
:1016F00009707D004F0578004F04BE000000060011
:101700000104E000050032000082FB0004024200F8
:10171000E580200065027A00040037000082FB00AB
:1017200004024200A580200065027A008002EB00DE
:101730000400E0001A00320012029800034A780008
:10174000144190000244B2001242980014419000EB
:101750000234A00012429800144190000274A000CC
:10176000124298000104E000070032000080FB00F4
:1017700000004000E1802000008040001020A20016
:1017800084027800060037000080FB000000400063
:10179000A1802000008040001020A2008402780078
:1017A00005007800000006000004E00014003A0084
:1017B00081C0B300B040800001487800B040800094
:1017C0002195200011009800C1C0B300114098007D
:1017D000B0408000904090000174A000114098003B
:1017E00041C0B300704080001140980070408000FC
:1017F000904090000174A000114098000000060085
:101800008180FB000080FB00000040000080400061
:101810004300DD0002A0200082014000134290003E
:1018200041C8B30001427200944198006400400036
:10183000020040001041900081407100114098006A
:101840000000060094A4AB00190032000080FB00E9
:1018500000004000E18020000080400090007800FF
:101860001103BE00040420000500200006036200EE
:101870008003EB008688BE00900078001103BE0054
:1018800084186B0085906B00900078000120A20006
:1018900001087800914190000344B2009340980001
:1018A000100078009040900004C168001240980039
:1018B000000006002048E2002A003A0010C0B300F1
:1018C00020E8B7002148E20026003A0021E8B700EE
:1018D00019C8BF00E24F50000A003A007040800073
:1018E0000048EB0081C4B3007040800011409800B4
:1018F00070408000904090000174A000114098005A
:1019000000000600E14F500016003A001E68EF008C
:1019100080C0B300A140800080487800A2408000D1
:10192000219520001101980043C0B3001341980095
:10193000A2408000924190000374A00013419800DF
:1019400014C0B300E381200084497800B2408000D5
:1019500000497800B04080001100980001C8B30031
:101960001140980000000600A0408000104278005E
:10197000414A8000C808DE00A09420001080FB00CF
:101980004800DD00008070008480FB00808F5000E4
:1019900001003600004278008480FB000100500006
:1019A000819420004801DD00F30F20009181610047
:1019B000828871004800DE008180E800804878005D
:1019C0000404E000090032000000EB0061942000F4
:1019D00011017800A3952000634978008208E8008F
:1019E0000000E800804F5200F8FF3E00414A8000AE
:1019F000C808DE00A09420001080FB004800DD0035
:101A0000008070001900320081C0B300B040800037
:101A100001487800A1952000B04080001100980096
:101A2000A040800010E8A30008003A0081C4B30081
:101A3000B040800011409800B0408000904090007D
:101A40000174A000114098000000060081C0B3009E
:101A5000B040800011409800B0408000904090005D
:101A60000174A000114098000000060081C0B3007E
:101A7000B040800001487800B040800021952000EF
:101A80001100980041C0B30011409800B0408000A0
:101A9000904090000174A00011409800514A8000CD
:101AA000C808DE00C09420001080FB004800DD0064
:101AB00000807000010032000000010080942000CE
:101AC0001070A1000148E20001003A0079FF070010
:101AD0000000060019C8BF00E24F500001003A00A4
:101AE000A1FF37001968EF001E48E2000D003A0020
:101AF00081C0B300B040800001487800B040800051
:101B00002195200011009800C1C0B3001140980039
:101B1000B0408000904090000174A00011409800F7
:101B2000000006001E68EF00000006000268EF00DB
:101B30000068EF0019C8BF00E24F50000D003A00E6
:101B400081C0B300B040800001487800B040800000
:101B5000A19520001100980081C4B30011409800A5
:101B6000B0408000904090000174A00011409800A7
:101B700000000600809520001080FB009195200059
:101B80009180FB00C808DD008100700040942000B7
:101B9000908F500007003100809520009080FB005E
:101BA0000000E8001081FB004811DD004094200097
:101BB000010871001FFC0700A19520007040800003
:101BC0001100980081C4B30070408000114098005B
:101BD00070408000904090000174A0001140980077
:101BE0000000060094A4A900000820002194200011
:101BF000110060001F003A00809420001004E000F3
:101C000008003D0020C0B30019E8B7000048E2001A
:101C100001003A00C5FF07002168EF002068EF00CF
:101C20000000060081C0B300B04080000148780089
:101C3000B04080002195200011009800C1C0B30081
:101C400011409800B0408000904090000174A000C6
:101C50001140980041C0B3007040800011409800CE
:101C600070408000904090000174A00011409800E6
:101C700000000600209520001004E0000A003D004E
:101C800010C0B30019E8B7000248E20001003A00B2
:101C9000A6FF07002168EF002068EF000148E2007E
:101CA00014003A0003FF370020C0B30019E8B70062
:101CB00081C0B300B040800001487800B04080008F
:101CC000219520001100980041C0B30011409800F8
:101CD000B0408000904090000174A0001140980036
:101CE0002168EF002068EF000148E20001003A009F
:101CF000F0FE0700000006001868EF000168EF0022
:101D00000268EF000068EF001E68EF001968EF003E
:101D100070408000904090000174A1001140980034
:101D2000704080000020A200704088009040900029
:101D30000174A100114098000E48AA00B040800034
:101D4000904090000174A100114098002094200060
:101D50000048EB008000EB00214A880080942000BE
:101D60008180FB00010878000080E80001F02F006E
:101D700010886000AEFD07000001EB0082007800D3
:101D800030002000AB02070096FF3700D0C2B3003E
:101D90001FE8B700C1812000914078000100780061
:101DA000B00FB20013003A00C10FB20000A0200033
:101DB00080804000A1408800010078000020A2003F
:101DC000B040880002C023001101610000402300E0
:101DD000800F510006003A0011009000219520006C
:101DE00007000900B05878008000B100C2FF37003A
:101DF00038FF3700E80F500001003A0052FC07009E
:101E00000000060010418000214180006100400078
:101E1000E080480010418800214188000448E20029
:101E200004003A000948EC0009E8B70001003A0054
:101E300009E8EF0000000600881F780030408000AD
:101E40000000E00012003A009424EF008C24EF0020
:101E50002000200030258800A824EF008644A90037
:101E6000F0092000802488006024880082C4A80033
:101E70009404AB0003003A009404A8009404AB005F
:101E8000FDFF3200100020003040880002003700C3
:101E9000E10F500008003A0094C4AB0006003A007D
:101EA0008AA4EF008C24EF008C04A8008C84A80086
:101EB00020002000304088008084AB000500320004
:101EC0008284AB000300320000012000002488005F
:101ED00066FC07008824AB00020032008EC0A90017
:101EE000690037008A04AB00070032008C04AB00A5
:101EF0000500320092FD07004000200030408800BD
:101F000010002000502488008A84AB0003003200B7
:101F10008C84AB00010032005EFC070080C4AB0083
:101F2000030032000004200000248800B5FF0700F1
:101F30008A44AB000E0032008C44AB000400320037
:101F4000120020008000EB0030072000390207005B
:101F500040002000502488001FC8BF00030032004A
:101F60000040E9001FE8B70001003A0051FE0700F9
:101F70008AE4AB00030032008CE4AB0001003200C5
:101F8000DBFB07008A24AB00090032008C24AB0085
:101F900007003200120020008000EB00F0FF270055
:101FA000240207008EA4EF002000200050248800A7
:101FB00030408000E30F500002003E008EC0A900B8
:101FC000310037008C64AB002E00320048C0B300F3
:101FD0008A64AB0003003A002A0037008A64AB0031
:101FE0002800320091248000C08120000148780040
:101FF0000181FB004411DE000240780002427800BB
:10200000D381200084497800820020005224880077
:102010000138A30009003A008080FB0002952000EF
:10202000E2C1780061C261000404A2000304A100BF
:1020300084C1710003F17800080037008080FB0044
:10204000E2942000E2C1780061C261000404A200B1
:102050000304A10084C1710003F178000004E000D2
:1020600002003A0049FF0700040037000001EB00BE
:10207000C181200020072000EE0107000844E9008C
:10208000D6FF3A008EC0A9004F0478000000060079
:10209000104180002141800000000600881F780068
:1020A0002628EF002828EF0090CAB3002AE8B700DE
:1020B00000802A00604188002000200070418800D4
:1020C00018C0B30008407800818320008848780059
:1020D0003068EF0034A8EF0036A8EF003268EF0058
:1020E000D1C1B30070FD070003C4B300028C20000F
:1020F0008040EB000840780081FD070030418800F7
:102100004F0478000000060012832000124178007E
:102110000281FB008001EB004A18DD00C610DE00E2
:10212000810070004A10DD0022042400023B880078
:102130008141780022032000034978000081EB00F0
:102140000208BB001000FC0050052000303B880056
:10215000A00A2000303B880061E7A80000000000D2
:10216000000000006007E200FEFF350000000600EE
:1021700030002400003B880032C8BF001D00320040
:10218000019020000081FB008001EB00A441800051
:10219000B54180000201520083815A000342780059
:1021A0002003200004487800020078001108BB00DA
:1021B000110190000288BB001000FC0050052000B7
:1021C000303B8800A00A2000303B880061E7A8006F
:1021D00000000000000000006007E200FEFF350084
:1021E00032C8ED0032E8B700E48040000004E000AF
:1021F000E4FF3A0061C7A9000000060023032000A5
:1022000093417800400ADE00050020000443780076
:102210002203200006497800000178001282BA00EB
:10222000840078001200BA000342780022032000E4
:102230000449780000000600889FBE008A9FBE0007
:102240003048E20022003A00404180000000E000F7
:10225000020032001000E0007301350030418000C0
:102260000000E00005003A00F08B2000F183200020
:102270000204200000014100030037001000E000CC
:10228000F9FF3D0068013700D0687800820F5000E8
:10229000FDFF3A0003C4B300028C20008040EB0035
:1022A00010C0B30016FD07003041880010C0B30015
:1022B00030E8B700F0872000010420008080400053
:1022C0000068EB00810F5000FDFF3A005601370017
:1022D0000084200010407800E54F5000910032004B
:1022E00006003E00E34F50005A0032006E003E00F0
:1022F000E24F50004C013A0006003700E74F500013
:10230000E6003200DB003900E84F500046013A0099
:102310003A01370020C0B3000188200080487800CF
:1023200082C3B3008100E800824878008100E800A1
:102330008048780011C0B300308820000148780040
:102340000040EB00418820008048780082C1B30043
:102350008100E800824878008100E8008048780029
:102360008100E8008048780000802E00F1FF2F00F7
:102370006241800073418000020040008380480079
:10238000F20F200083882000824960004802DE00AE
:102390008301E800844978008301E80082C9600075
:1023A000C808DE000300E800014878000000E800EB
:1023B00000C8EB003848E20019003A0031C0B30011
:1023C000014878000040EB0082CFB300E380410079
:1023D00082487800B2CAB3008100E80082487800E1
:1023E00022C0B3008100E800824878008100E80044
:1023F0008048780082C0B3008100E80082487800FD
:102400008100E800804878008100E800804878007A
:102410008100E800804878000100E80000C8EB0077
:10242000404180000000E000020032001000E000A7
:10243000FD00350003C4B3000288200011C0B300C2
:1024400001407800AEFC0700404188003068EF0092
:10245000F5003700108420001004E00008003A0066
:10246000A0CAB3002AE8B70083BF2A0063418800EE
:1024700023002000734188003868EF00080037000F
:1024800090CAB3002AE8B70000802A0060418800A3
:10249000200020007041880010C0B30038E8B70069
:1024A0003068EF00E00037008000EB0010002000F3
:1024B00010010700C05928005601070060C0B30092
:1024C00031E8B7002AC8BF000080FB000000E80028
:1024D000E60F50000B0034000BFF070056FE07000C
:1024E0003148EC0031E8B7000080FB00A1822000F9
:1024F000914078008180FB008100E800810F50004E
:10250000F5FF350061C7A9003068EF008000EB00DF
:1025100010002000F7000700E05A28003D010700E6
:10252000C1003700A0418000B1418000E10F4000B0
:10253000E08F48000E003A00128420001281FB0058
:10254000238420009381FB00C819DD000300710083
:10255000328420001281FB00438420009381FB0021
:10256000C819DD0083007100A0418800B1418800D6
:10257000128420001281FB00238420009381FB0041
:10258000C819DD0003007100328420001281FB00B5
:10259000438420009381FB00C819DD008300710093
:1025A000A2418000B3418000820F5000838F580009
:1025B0002E003A005084200010407800E14F500077
:1025C0002A0036000044EB0021832000914078006F
:1025D0000181FB00820141000080FB00820320009A
:1025E000000051004F01DE00000041000081D100D9
:1025F0000880FB0000004100640040000000400033
:1026000002842000624278000482FB000000410046
:10261000104190004811DD0002017200009020007E
:1026200002B079000140E80032E8B700A241800022
:10263000B341800061014100E0814900A24188006E
:10264000B3418800FC4F500001003A00C8FE07006B
:102650000844E80050842000104078008080FB008F
:102660008100D100814F5400D7FF39003068EF005E
:102670006D003700BEFE070034A8EF0036A8EF005B
:102680003068EF008000EB00100020009900070088
:10269000D05B2800DF000700630037004041800066
:1026A0000000E000020032001000E0005E00350093
:1026B00071C0B30000882000014878001284200017
:1026C0001281FB00238420009381FB00C819DD00E8
:1026D00003007100328420001281FB00438420003B
:1026E0009381FB00C819DD0083007100F20F200008
:1026F00013882000824960004802DE008301E80060
:10270000844978008301E80082C96000C808DE00BF
:102710000300E80001487800508420001040780051
:102720008380E80080487800E14F50002B0036009D
:102730000044EB000881FB008001EB0014842000C2
:102740001482FB00258420009582FB00C82ADD004E
:1027500005007200348420001482FB0045842000B0
:102760009582FB00C82ADD0085007200020040004F
:1027700083804800A1FE07008884FB005484200069
:102780009482FB008502D1008583FB0007855400FD
:102790000A02B000068820000A0545000A05430029
:1027A000F40F2000044D6000C805DE001B459800B2
:1027B00081016200078054001002B0000000400058
:1027C0000000430004C86100C818DE0011409800F2
:1027D00008C4E80088CF5200D6FF3E0003C4B3000F
:1027E0000288200011C0B30001407800C4FB07003C
:1027F000404188003068EF000B0037008000EB009C
:10280000100020003B000700805D280081000700C9
:102810009424EF000080EB00000000000000E900BD
:10282000FDFF3A000000FE004F05BE004F04BE0051
:102830000000060031072000810F50000D0032001B
:1028400005003C00E10F500010003200E30F500083
:1028500011003A000F00370041072000810F50009F
:10286000080032008100E800810F50000A003A00A1
:1028700002003700FE00070007003700FC000700D9
:1028800005003700FA0007000300370003FE0700C9
:10289000010037007100070010000500EC22A800BD
:1028A000000000000000000000000000EC22A90071
:1028B0000000060000F02F00E022B600F002A900A0
:1028C000F022A900E822A900F402A900F422A9003C
:1028D000EC22A900000006000000FB0001F02F0020
:1028E000221780008280600080807000211788009D
:1028F0000000060080417800F00F2000E022B700C1
:10290000F422A800F402A900EC22A80000000000B4
:10291000000000000000000012178000EC22A90057
:102920000278A300F8FF3A0002F02F00002E2000EA
:1029300010086100F422A9008180FB008100EA00F8
:10294000CF08DE00A21780000200A1000281700003
:10295000A217880003407800DFFF0700CFFF370091
:10296000D4FF070000202100A10720001801070064
:102970008040EB0080C3B300DEFF07008040EB0027
:1029800080C0B300DBFF07008040EB0010C0B30045
:10299000D8FF07008040EB0060C0B300D5FF070000
:1029A0008040EB00C0C0B300D2FF070000B82B008E
:1029B0000100200006013700F0F32F004427B60085
:1029C00042A7AB0003003A000000000042A7AB00A2
:1029D000FDFF320040A7A900F0C2A900D022A80044
:1029E000DFFF07000000EB00E3000700D4FA070058
:1029F0000060FE0010FD070030408000FF0F500017
:102A0000FBFF36008824AB00F9FF3A000AFE0700FE
:102A1000F7FF3700881F780000047800184078001E
:102A20000004E0000B003200EA4F500004003A00BE
:102A30008040EB0000CCB300AEFF0700020037007F
:102A400011C0B300ABFF0700584078000004E0005D
:102A5000F5FF3A004F0478000000060020952000A2
:102A6000104078007F406000E14F500054003A0071
:102A7000609520001004E00051003A00630050000F
:102A800061C0B30090CF10001B003A000080E80046
:102A900010407800FBC04000814F5000040032001D
:102AA0008140E800814F500013003A000B003700CE
:102AB00008C8BF00E14F50000F003A000050280046
:102AC000004A880090002000204A880001CCB30012
:102AD0002094200001487800070037006057280044
:102AE000004A8800D0012000204A880001CCB300B1
:102AF00020942000014878002095200002C6B300F1
:102B00009040610000C2B30080CF50002C003A001A
:102B10003095200010407800E34F5000190032003B
:102B200003003E00E24F500025003A000500370048
:102B3000EA4F50000B003200EB4F500020003A00EB
:102B400018003700A0832000004A880010002000F1
:102B5000204A880011CCB30020942000014878005E
:102B60000000060001C8B30020942000014878004E
:102B70005095200010417800A18320008248780001
:102B800000000600B0832000004A880010002000EA
:102B9000204A880011C8B300209420000148780022
:102BA0000000060001C8B30020942000014878000E
:102BB0004095200010417800B183200082487800C1
:102BC00000000600E10F500003003200E20F500049
:102BD00004003A0002003700F4C2A800000006001A
:102BE000F4E2A80000000600E10F500003003200EC
:102BF000E20F500004003A0002003700F4C2A900BE
:102C000000000600F4E2A90000000600E10F5000F9
:102C100003003200E20F50000B003A0005003700BD
:102C200000042000F402B6000000EA004F00DE00BD
:102C30000000060000082000F402B6000000EA00D0
:102C40004F00DE000000060000000500E10F50000C
:102C500003003200E20F500004003A000200370087
:102C6000F0C2A90000000600F0E2A9000000060082
:102C70008824AB000200320010002000DAFF370089
:102C8000000220000608E30010003A00F041800036
:102C9000E10F500002003A00CAFF07001A00370097
:102CA000B1042000810F500003003A001000200002
:102CB000CDFF07001400370061092000810F50008C
:102CC000110036003E28EF000F003700F041800071
:102CD000E10F500002003A00BAFF07000A00370077
:102CE00021032000810F500003003A001000200053
:102CF000BDFF070004003700613B2000810F50003A
:102D0000010036003E28EF003E28EC0000000600DF
:102D10004009000022000000000000000008000040
:102D20002600000000000000000A00002000000053
:102D3000000000003A08000002000000000000004F
:102D4000400800000001000000000000260800000C
:102D500014000000000000003C0800000200000019
:102D600002000000010000003E0800000200000018
:102D700000000000000000000000E00013003A0026
:102D800083E0A800100020002700070010002000AA
:102D90001D0007000004E00006003A003008200093
:102DA0004007B6000300320083E0A900001A0400C7
:102DB00000000000E05D280016FF07001000200062
:102DC000A2FF070020002000A0FF0700000006006F
:102DD000F03FB1000180B10006003500EE030900AC
:102DE00000000000403FB1000180B100FBFF3D004A
:102DF0001000B000203FB000020035000080090044
:102E00000000000000000600E10F500005003A003D
:102E100090168000620060000000E9004F00DE00B4
:102E20000000060000000500E10F500001003A001C
:102E3000D022A80000000600FFFFFF00FFFFFF00F8
:10340000101B040000000000B01C040000000000BD
:10341000B01C040000000000B01C0400000000000C
:10342000B01C040000000000B01C040000000000FC
:10343000B01C040000000000B01C040000000000EC
:10344000B01C040000000000DC1B040000000000B1
:10345000B01C040000000000B01C040000000000CC
:10346000B01C040000000000141C04000000000058
:10347000B01C040000000000B01C040000000000AC
:103480007E1C040000000000B01C040000000000CE
:10349000B01C040000000000B01C0400000000008C
:1034A000B01C040000000000B01C0400000000007C
:1034B000B01C040000000000B01C0400000000006C
:1034C000B01C040000000000B01C0400000000005C
:1034D000B01C040000000000B01C0400000000004C
:1034E000B01C040000000000B01C0400000000003C
:1034F000B01C040000000000B01C0400000000002C
:10350000B01C040000000000B01C0400000000001B
:10351000B01C040000000000B01C0400000000000B
:10352000B01C040000000000B01C040000000000FB
:10353000B01C040000000000B01C040000000000EB
:10354000B01C040000000000B01C040000000000DB
:10355000B01C040000000000B01C040000000000CB
:10356000B01C040000000000B01C040000000000BB
:10357000B01C040000000000B01C040000000000AB
:10358000B01C040000000000B01C0400000000009B
:10359000B01C040000000000B01C0400000000008B
:1035A000B01C040000000000B01C0400000000007B
:1035B000B01C040000000000B01C0400000000006B
:1035C000B01C040000000000B01C0400000000005B
:1035D000B01C0400000000005A1C040000000000A1
:1035E000B01C040000000000B01C0400000000003B
:1035F000B01C040000000000B01C0400000000002B
:10360000B01C040000000000B01C0400000000001A
:10361000B01C040000000000B01C0400000000000A
:103620002FAA20000E7F24000E0188000000000059
:10363000000020000000E000020032000001200035
:103640002002880014000700C70007000000E00007
:1036500003003A00C08A2500010020000200370064
:103660000000200001002000810F700001003200E6
:1036700014000700000020000000E00002003200FB
:10368000000002000000000096460200000000005A
:103690000040DA000000FE004440A9002010200095
:1036A0000000E0000300320000002000A0018800BC
:1036B0004440A800000006008A1F78008B1F780095
:1036C0000000060091018800800478000000EB00F3
:1036D0001A003700E284440032A0B4009905BA0011
:1036E000E284440032A0B4009906BA00E2844400A7
:1036F00032A0B4000006EB00476FDE00FD07B20009
:10370000636CE10003003A00EBFF07000000EB00F0
:103710000A003700606CE10004003A00005DEB0035
:103720008B05E900FDFF3E00040037006168E10001
:10373000010032000086EB000B00070019C7BA0039
:103740001905BA000E04E00003003A000A00E00088
:10375000E0FF3A0000000600FE07B2009E0188006C
:103760008A047800F5FF3700395DBA008B05E9005F
:103770000C003200295DBA008B05E9000800320018
:103780000C00E00003003A00E284440032A0B400E0
:10379000F5FF370019DDBA008B05E900FAFF3A00A2
:1037A0008904E800E184440032A0B400000006006F
:1037B0003C20040000000000809FBE003400F800A0
:1037C00000002000A00188000000FA0061178000BE
:1037D000000220000080600000F0A7000000EA0066
:1037E0000000E9004F00DE00004078000080FB0090
:1037F000610060004500DD00611780000150A100FC
:103800000100700060178800A0088000404E88000A
:103810001421EF008460A9000080FA003400F90050
:103820004F00BE0000400600809FBE003400F8003C
:1038300000002000A00188000000FA00E0168000CF
:103840000080EA004F00DE00004078000080FB00AE
:103850004F00DD00E116800001F0A10001007000C2
:10386000E0168800E116800000002400008060005F
:1038700000F0A7000000EA000000E9004F00DE00B1
:10388000004078000080FB00610060004E00DD0019
:10389000E116800001E0A10001007000E016880040
:1038A0008500A9000080FA003400F9004F00BE0036
:1038B000004006003600F800809FBE00829FBE00D8
:1038C000849FBE00869FBE003400F80000002000E8
:1038D000A00188000000FA00520D07000080FA00E5
:1038E0003400F9004F03BE004F02BE004F01BE007E
:1038F0004F00BE003600F90000400600809FBE0069
:10390000829FBE003400F80000002000A001880063
:103910000000FA00DDC8BF008081FB00311180008B
:1039200001417800D18C20008180410082487800DC
:103930000040E800DDE8B700DDC8BF00F04F5000F0
:1039400001003A00DD68EF008560A9000080FA0000
:103950003400F9004F01BE004F00BE0000400600D9
:103960000040DA000000FE000000050003F0A200A5
:10397000889FBE008A9FBE008C1F78000901070047
:10398000100133006450E1004F0032006420E10078
:103990005200320003826C0007003B000905D00092
:1039A0000306D000820F54000C065D0002003900AF
:1039B00002003200890178000306780085825500F4
:1039C00004003D000003FD008103FD008502EA00C4
:1039D0008B854200840F720002003B0060001000E3
:1039E000E08018006011B8000005EB007A28E100C3
:1039F0000A00390006007800C75DDD00F707B20055
:103A0000878075002D003700828171000A017800DF
:103A1000610560008180D1000080D3008502E9004B
:103A2000F9FF3B00060440008784480002003B0089
:103A300060041400E0841C000988A3000700320021
:103A40008A81710082817100610164008904D10062
:103A50000884D3008B05E800170037000978A3001D
:103A600013003A000B00E000130034008B05E9005E
:103A70000804440089844C000A4474000978A300B7
:103A80000D003A000B00E000070034008B05E90050
:103A90000804440089844C0001003A000B00200017
:103AA0000978A300F7FF32000001EB0002003700A5
:103AB000828171000A0178007F0007000CF0A700E6
:103AC00001F0A000C80037006420E10002003A00C5
:103AD000838F6C00C80033000801BE000200BE00E6
:103AE000C1003700889FBE008A9FBE008C1F7800EF
:103AF000AC000700B300330003866C006450E100A3
:103B00002E0032006420E100330032006150E100F9
:103B10002F0032006120E100310032008585550020
:103B2000EB07B00009002000080420000500370062
:103B30000804440089844C000A0031000603430055
:103B400087834B000001530081815B00F8FF330045
:103B50000203BE000800A0000804440089844C0051
:103B6000F6FF3900C639DD00830173000100320021
:103B7000130020008904D1000884D3000998A30011
:103B8000050032000800A7000300A0008904D1004E
:103B90000884D3008B05E8008904D1000884D30091
:103BA0000001EB000281D2004300070001F0A100F8
:103BB0000CF0A70001F0A0008B0037006420E100AA
:103BC0008D0032000801BE000200BE00F7FF370082
:103BD0006120E100880032006000B800F3FF370088
:103BE0000000200001F82700F0FF3700839F6800E5
:103BF0000100E00002003D0060001000E0801800BD
:103C00000300E00002003D0060011100E0811900A6
:103C1000B00007004F00E00002003B006000100011
:103C2000E0801800000006000001BE004800070008
:103C30000470A70003F0A1006509B100160032006E
:103C40000D0035006828E10006003500F0FF2F0068
:103C5000F1FF27000300E00013003B0001002800F3
:103C60000000050000004000818048008502E90056
:103C7000FCFF3A0008003700F88F420002003C00C9
:103C80008000EB00000005008100D1000080D3001F
:103C90008502E800FCFF3A000300E00002003B0060
:103CA00060001000E0801800000006004F89DE0070
:103CB0008201780097003700810020006180550064
:103CC0000B003D000B00200061FE2F000100E10011
:103CD0001D00340082817100610164008904D100FB
:103CE0000884D3000000E800FAFF3A0071002000C9
:103CF00061006400030070000200600009003200EF
:103D000061044400E0844C000988A50005003200ED
:103D10008B05E8006808E10002003A008904D10040
:103D20000884D300F20F20000258E10005003D0096
:103D3000C75DDD00F907B2008980750008007800D2
:103D4000000006000BF827008B007800000005003B
:103D5000C70ADE00F107B200F50FB200080032001A
:103D6000E1CF4200020032000170A00024000500F3
:103D7000810F7000010032000408050044000500B6
:103D8000810F700002003A00140005008502E9006E
:103D90000000400081C04800FCFF3B000170A00013
:103DA000240005000004BE00E9FF07000003BE0078
:103DB0000405BE000200BE00E5FF0700844F750049
:103DC000000006000200BE006450E100050036005D
:103DD0006420E100020036000968A30001003A00F7
:103DE0000800BE000160A0004F0678004F05BE002D
:103DF0004F04BE0000000600F0FF2F00F1FF270077
:103E0000F9FF3700889FBE008A9FBE008C1F780094
:103E1000E4FF0700EBFF330003866C006450E10011
:103E2000240032006420E100270032006150E100EC
:103E3000220032006120E100210032008B85420027
:103E4000EB07B1000134B800003AB80008044200A2
:103E500089844A00013AB8000030B80088804000E8
:103E600009014A000400330000004000818048003E
:103E7000020149008B05E900C909DD0083017000DA
:103E80000100320013002000C814DE004814DD00D9
:103E90004709DE001200B200C808DE000884700086
:103EA00085FF070001F0A1000CF0A70001F0A000C1
:103EB000CDFF37006120E100CFFF32000801BE00D6
:103EC0000200BE00F7FF37006150E100FCFF3A003E
:103ED000C9FF37006022B800060220000000D000B1
:103EE0008180D2000482D2008582D2000000A0002E
:103EF0000202520083825A00030031000202420093
:103F000083824A000000A1000603E900F3FF3A00A3
:103F100000000600881F7800030478000300E0001A
:103F200007003D0060001000E080180060011900EB
:103F3000E081190002003B0001F02D000300370072
:103F40000400070008F0A70001F0A0004F0478006B
:103F500000000600889FBE008A9FBE00008270009D
:103F60000402710004827100260032000004BE00C9
:103F70000200BE006011B8006B092000950220000D
:103F80000182CF000A0039000541B1000082CF0054
:103F9000070039000541B1000982CF000400390053
:103FA0000541B1000882CF00010039000541B10090
:103FB00005425200120032000A003B00828171006B
:103FC000610164008100D1000080D3008984D300A6
:103FD0000884D3008B05E8000442E800F7FF3A00AC
:103FE000070037000804440089844C0000004800A2
:103FF000818048008B05E9000442E900F9FF3A009E
:104000002DFF07004F05BE004F04BE000000060054
:104010008001780002003700B15978000201E90000
:104020000200E000FCFF3A0000000600800178007A
:1040300002003700815978000201E9000200E00027
:10404000FCFF3A000000060000017800B141780052
:10405000035978000304E000FCFF3A00000006006A
:1040600080007800010178003104E000FDFF3A0093
:104070000000510000000600881F7800020478004C
:1040800008017800E2FF0700080040004F047800B4
:10409000000006000000FA00881F78000004780085
:1040A000EA8157003FB9970088007800C0032200DA
:1040B000070007000000E000020035008040EB0030
:1040C000017478004F0478000080FA0000000600B8
:1040D0006200FA00889FBE008A1F78000005780001
:1040E00081047800020478008300780080F92F00B2
:1040F0000F004000680607009A979F00A9979F004D
:104100000000EB00B09F9F001885FB008A04FB00B5
:104110000A05EA004F55DE0050022000808F54004F
:104120000D003200E10F55000B003A000A01780043
:10413000880078002F9097009F919700030001005E
:10414000A0979F000000E0008E0032003F9897008B
:104150000000E800B09F9F000A04440050022000C5
:10416000808F5400040032000900E000E6FF3A00AE
:104170003F989700840037000000EB00909F9F005D
:10418000809F9F00F0979F00E0979F00D0979F002F
:10419000C0979F0007003700C1A920000100500010
:1041A0000000400001A9200061007800DF9897001E
:1041B00001007000D09F9F008804780009047800F7
:1041C000384578008A00FB00C0A9200011040700D0
:1041D0000000E000F0FF3A00A1C2B300814F55009B
:1041E0000E003A00CF8897000180E900C08F9F0041
:1041F00010007800C09F9F000000E00005003D0017
:104200000000EA00C09F9F005F9897000020A00078
:10421000D09F9F000904E8000F003700C09F9F0057
:104220000000EB0005003700F2FF2700820F50006E
:10423000020032006A01B9000280400009047800DF
:1042400088047800B900FB000103B100E98F500039
:10425000F5FF3600C09F9F00E0C2B300984F1000EA
:10426000020032000080EB0019003700A0C2B3004A
:10427000D84F100007003A00CF8897000180E9006E
:10428000C08F9F0010007800A09F9F000804E800E6
:10429000100037000000EB00A09F9F00880078000E
:1042A00005003700F3FF2700830F500002003200A3
:1042B0006A02B90004004100010478008800780017
:1042C0003101FB000203B100E90F5100F5FF360098
:1042D000A09F9F00984478008900FB0080A82000E0
:1042E000CC0307000000E000020032000804E800F0
:1042F000010037008044EB00C97F9F0080C6B300F7
:1043000080CF540004003A0098CF14000A003A000D
:104310006640500006003700C0C6B30080CF54008E
:1043200005003A0098CF140003003A0065404000B1
:10433000C07F9F000804E8001801FB00E3FB2F008A
:104340008F81410081F92F008F804000A0F92F005C
:104350000F004000100007000000E00009003A00D4
:10436000E1FB2F008F804000A0F92F000F004000DC
:104370000D0507000000E000020035000804E80019
:1043800061FF37000080EB004F0578004F04BE004E
:104390000080FA0000000600889FBE008A1F780097
:1043A00000047800824478000305780070C6B300EA
:1043B00080CF54001A003C0000C0E90080CF5400B8
:1043C000CD003D006D40500080CF5400770032009A
:1043D0000B003C007140500080CF540035013C0080
:1043E00000C0E90080CF5400C3003D0050C2B300BC
:1043F00080CF54002C0132007C4040000500370083
:1044000030C6B30080CF54001A0032001E003C00BA
:1044100000C0E90080CF540026013A00B600370002
:10442000F0C6B30080CF54006000320007003C00AB
:104430006640500080CF54001300320065404000B9
:1044400080CF54001B013A00D400370050C7B3009E
:1044500080CF5400550032006340400080CF5400AC
:104460005200320002C7B30082CF540011013A005B
:10447000FF0037001181E900820878007800900081
:10448000127578001101370028609000C2C6B30091
:10449000824F500007003A0011017800640051007B
:1044A000800878001000BE004F89DE00820178008D
:1044B0001400370012C7B300824F500003003A00C7
:1044C000110278006800520005003700A2C6B30050
:1044D000824F500006003A00910278006880520036
:1044E000800878005001BE004000BE000500370083
:1044F0001180E9008008780010007800CF80DE008D
:104500006109B900009CBE000294BE0028629000C0
:1045100085C6B300854F52000D00320025C6B3009A
:10452000854F520004003A000000FB00CF80DE00FF
:104530006109B9000800370045C7B300854F520034
:1045400003003200E6C24200854F520004003A00E8
:10455000CF80DE006109B900009CBE000294BE005D
:104560003802BE002803BE0078009000D1C2B3001C
:10457000E00F5200E08F5A00E00F5B00E08F5B001D
:1045800008003500881090000118A30002003200D6
:10459000B1C2B300030037000108A300510032008C
:1045A00001C2B300017578004C003700286090000C
:1045B000C2C6B300824F500008003A0011037800D1
:1045C00064005300800878001002BE006033B80019
:1045D0000400BE000601BE001400370012C7B3007D
:1045E000824F500003003A00910278006880520028
:1045F00005003700A2C6B300824F500006003A0003
:104600001103780068005300800878005001BE0054
:104610004000BE00050037001180E90080087800E6
:10462000100078008000EB006011B800009CBE0014
:104630000294BE002862900085C6B300854F5200E8
:104640000D00320025C6B300854F520004003A0029
:104650000080FB008000EB006011B800080037000C
:1046600045C7B300854F520003003200E6C2420046
:10467000854F520004003A008000EB006011B80042
:10468000009CBE000294BE00081090000038A300F9
:10469000140032003800BE002801BE00E00F5000B8
:1046A000E08F5800E00F5900E08F59000D003200F4
:1046B00080C7B30080CF54000300320080C5B30030
:1046C00080CF540007003A007800900001C3B30087
:1046D000017578000000E800097578000000E80026
:1046E0007004980078009000000545006A04980066
:1046F000894078006900370028619000C0C4B30089
:10470000804F510006003A00910378006880530002
:10471000800878005001BE004000BE000500370050
:104720001101780064005100800878001000BE007C
:10473000D0050700009CBE000294BE00B8009000A7
:10474000780090000100E00002003D00D1C2B300FB
:1047500008003700881090000118A3000200320002
:10476000B1C2B300030037000108A3000400320007
:1047700001C2B300017578000000E80070049800E1
:1047800078009000000545006A0498008900FB004D
:1047900008007800530007004E00370028619000A1
:1047A000C3C6B3001180E900834F510024003200DA
:1047B0000A003C00E4C15100834F51002700320041
:1047C00083C1E800834F51001500320020C6B300BA
:1047D000804F510020003A000A00370043C7B30061
:1047E000834F51001D003200E6C14100834F51004C
:1047F0001A00320010C7B300804F510016003A0073
:10480000060037001180E900800878001000780069
:10481000485C9000084878002E0037001180E900BD
:104820008008780010007800680A9000CFA2DE00AF
:10483000612BB9000498BE000690BE002500370029
:10484000800878001000780068099000CF91DE00A1
:104850000288BE001F0037001180E9008008780040
:1048600010007800680C90000808780019003700E4
:104870001181E9008208780012027800CFA2DE00E0
:10488000612BB900049CBE000694BE00F8009000A5
:10489000010545006A04980080407800080078000F
:1048A000920207000B00370078009000097578002D
:1048B0000600370078009000000545000904E0007C
:1048C00001003A0059C2B300094D78000000E80029
:1048D000700498000000EB004F0578004F04BE0004
:1048E000000006002F04B000889FBE008A9FBE0013
:1048F0008C9FBE008E1F78000007780081F79F0014
:104900003E04BE002E05BE005E0890000000E000E0
:1049100002003D0060002000500F98008E007800DB
:1049200020FB2F000F00400046020700E20F50005E
:104930000A003A0030002000100F9800B1C9B300FF
:104940000FF097008140400040A32000E1CF5000CD
:104950000D003E0000A320000B0037000000E00027
:104960000F00340030002000100F9800B1C9B300D0
:104970000FF1970081404100C0A32000E1CF50001B
:1049800001003E0080A32000EE009000B0487800B7
:10499000B06878001040780090409800F30037002D
:1049A0000000E00005003A0022FB2F000F0141004B
:1049B000001978008001EB00E70037006022B800A2
:1049C0006033B8000800BE000A01BE008004070082
:1049D0000000E00001003D000BF0A200705927002C
:1049E0009F9897000088B900026A280013002000F1
:1049F0007EFC0700640650009C9F9F0013003B0054
:104A000063061600C0FF2F00000666008C01EA0056
:104A1000939F9F000DA420000800BE000A01BE0065
:104A2000070037000C08A300030032003D02BE005F
:104A30002D03BE005E0507000C86D100E886460007
:104A40000C00E000F7FF3C00180037000C00E0000D
:104A500018003200C0FF2F00000666009C9F9F00D8
:104A60000DA420006000B8000200200003FF230016
:104A7000070037000C08A300030032003D02BE000F
:104A80002D03BE004A0507000C86D100E8864600CB
:104A90000C00E000F7FF3C000002BE000203BE0075
:104AA0000800BE000A01BE00530407000004BE0057
:104AB0000205BE00DE08900060C6B3000FF297004A
:104AC000804F5200040032006000200062C4B30036
:104AD000824F520002003A009F9A97006A8042007B
:104AE00081004000F1B79F0001037800F30F5300ED
:104AF0000200340037012000F7B79F0000C3B30065
:104B0000C0779F0056FB2F000F0343000E00780074
:104B1000A0B79F00060778003D0037000800BE00E0
:104B20000A01BE00F20407000006BE007FB1970034
:104B300068015100F2B79F004240A9000C00340008
:104B4000170507000002BE000203BE000800BE00F9
:104B50000A01BE008C0507006022B80046782D00CF
:104B600077192400120507000004BE000205BE00EC
:104B7000E80047008E0020000802BE000A03BE00C5
:104B8000B4B79F00C5B79F00D6B79F00E7B79F0097
:104B90000C01BE00010478000C003700A4002000C6
:104BA00005002000C0FD2F000F0040008401070019
:104BB0006FA89700FFA897000FB197009FB19700CB
:104BC00005C3B300056441000001BE00E00F5100C1
:104BD000E08F5900030034000E07E900E10F4700A1
:104BE000EEFF3A00880078003FB49700CFB49700FA
:104BF0005FB59700EFB597000200370000C3B30020
:104C0000806078000E07E900FCFF3B0068874000E9
:104C10007FB397000600E000070034006022B80070
:104C20006033B8000800BE000A01BE00ED030700B3
:104C30000000E000B9FF3C000E0378002FB797009A
:104C400051FB2F008F804000010353009F9B970072
:104C500067804300909F9F00020037000603E90031
:104C60000000E900010178008200780003C3B3006E
:104C7000B1CF1100F9FF3200909F9F00DE09900034
:104C800061C6B3000FF29700814F5200030032005B
:104C900061C4B300814F520002003A000000E800F6
:104CA0000A0037001000200051C6B3008FF29700B1
:104CB00081CF5200050032000540780050C4B20098
:104CC0000080FB000000E9004F00DE00830140008F
:104CD000868F510001003400860178000300E00057
:104CE0001D00350000C3B300868F510006003D0053
:104CF00062C279006940400041C3B300814F520055
:104D000001003C00694050008300E900810041003F
:104D100001003700840178000302E90001037800F4
:104D2000A142780080CF5200FAFF320091C3B30055
:104D3000814F500001003A00054BE8000400E000FC
:104D400005003D000201E9008301E8001F9B970078
:104D50000603E800969F9F008FF397008700FB00F3
:104D60001F9A97000E007800060007004F07780092
:104D70004F06BE004F05BE004F04BE002F04B10019
:104D800000000600F0874700889FBE008A9FBE0093
:104D90008C9FBE008E1F780000047800814478004C
:104DA0000205BE00040678000B00E00002003C0093
:104DB0001B0020004A9F200060C6B30080CF540033
:104DC0000E00320060C4B30080CF54000B003200EC
:104DD00070C6B30080CF54000300320070C4B3002B
:104DE00080CF540081003A00E40F46007F00350078
:104DF00058089000800F56007C003D000C06E8002B
:104E000060C6B30080CF54001000320060C4B3000D
:104E100080CF54000D003200081090000038A3002D
:104E200004003A0058089000808F550001003D00B2
:104E30005B0C9800580890000C005000500C980033
:104E400002003B000000EB00500C98001808900096
:104E5000E80090000C00E00026003C0002C3B30014
:104E6000827078000000E800100C9800D8089000CC
:104E70000100E00003003C00881090000138A3000E
:104E800005003200E8009000E2C2B30082707800B2
:104E90000000E800100C9800580890008C00EA0010
:104EA000810F500001003D000006EA008C00EA007E
:104EB000210C9800000646005C0C98008B0F5600F1
:104EC000010034000B0678003C0C9800E8009000CC
:104ED00018089000008040000C0178008A007800DB
:104EE0004BFC0700580890000C0650004C0C980032
:104EF000900037008C8F550018003D000080400066
:104F00000B0178008A00780041FC07001808900027
:104F100000804500100C98008B0556002B0C980063
:104F2000D80890000100E00003003C0088109000C9
:104F30000138A30006003200E8009000E2C2B3008E
:104F400082707800380890000000E800300C98006B
:104F500058089000400C9800760037000080400010
:104F60000C0178008A00780029FC070018089000DE
:104F700000004600100C98008C855500D808900061
:104F80000100E00003003C00881090000138A300FD
:104F900005003200E8009000E2C2B30082707800A1
:104FA0000000E800100C980058089000808F550011
:104FB0000100340080057800E80090001808900097
:104FC000008040008C0045000B01780010FC0700B9
:104FD000180890000B004000100C98005808900032
:104FE0008B0550002B0C98005200370018089000D9
:104FF000E80090009A7078000000E800100C98001B
:10500000D80890000100E00003003C0088109000E8
:105010000138A30005003200E8009000E2C2B300AE
:10502000827078000000E800100C9800580890008A
:105030000000E000100034008B05E900808F55006F
:105040000100340080057800E80090001808900006
:10505000008040008A00E8000B017800ECFB0700AC
:10506000180890000B004000100C980058089000A1
:105070008B0550002B0C9800E80090001808900059
:1050800000804000095878000007E8000C00E000AC
:1050900004003500B1C2B300014878008E047800E6
:1050A00004003700D1C2B300014878008E047800B4
:1050B0000C06EA007D8557008006EB0009003700EA
:1050C000A20020008C007800728057003100070099
:1050D0007FB097008FB89700016D780000067800C8
:1050E0008D06E8000C00E000F5FF3C000D00E0003C
:1050F00009003A008E04780000C3B300805C780099
:10510000050037008D06E900FC80570061C07E0075
:1051100002C3B300825C40000D00E000F9FF3C00D8
:10512000E80090001808900000804000808454003F
:10513000390C98000810900074006000F00F5000C7
:105140000E003A009808900078009000008040001F
:10515000A808900001004000B8089000010040003D
:10516000C808900001004000F8089000810F50002E
:1051700002003D0000805000000C98004F077800AE
:105180004F06BE004F05BE004F04BE000F01B10028
:105190000000060080027800010378001100090079
:1051A0000203D80080017800830A78000299B900D0
:1051B00002015300920298000500780000000600EA
:1051C000881F78008A9FBE008C9FBE000004780074
:1051D0000205BE000406BE000401BE000A00BE00B7
:1051E00082FA0700008CBE000C01BE00EB03070032
:1051F0000005550081855D002A0498003B04980055
:10520000080078004F06BE004F05BE004F0478002E
:1052100000000600020037000304E0000600320030
:105220000001780002007800B041780081CF510081
:10523000F9FF3A00010037000001EB00020078009E
:1052400000000600889FBE0000047800E68440004D
:105250001900D0004500DE00F27F2000820F5000D0
:1052600010003A00000CEB00990478006F81640094
:10527000200020001B003A00210190000200E00005
:1052800018003A00110190000200E00015003A00F9
:10529000100020001100E000120032002000200069
:1052A000100037000000E00004003A000100780020
:1052B000FB0107000000E00008003C00F2002800AD
:1052C0001901610001FE2300810C710021C02F0033
:1052D000010C40000080EB0002003700000CEB00E6
:1052E0000000EB004F04BE0000000600FC874700F2
:1052F000889FBE008A9FBE008C9FBE008E1F7800D4
:105300000006780080C5B30080CF50000A0032004C
:105310007740400080CF50000A00320069404000D2
:1053200080CF50000B003200309E200080BF9F00D5
:10533000AE0020000A003700229D200082BF9F009F
:1053400006003700339E200083BF9F008E002000A0
:1053500003003700349E200084BF9F000E01200010
:105360003C02BE002C03BE000605BE000404BE00C5
:1053700040C6B30080CF50000300320065404000BB
:1053800080CF50000B003A00E00F5200E08F5A002F
:10539000E00F5B00E08F5B0006003D006000B8009E
:1053A0006011B800040450008584580006055900B7
:1053B00087855900E80F57000400320040002000A4
:1053C000F00F570038003A0001003700300020008D
:1053D000E00F5400E08F5C00E00F5D00E08F5D00A7
:1053E00004003A00DC0890008D0120000100E0007C
:1053F000060032008E00E900888060008FBA9700B6
:10540000E5C07800F1EF9F007D012000800078006A
:105410008100E900050033008B05D1000A85D30027
:105420008984D3000884D300F9FF3700089EBE00AA
:105430000A96BE00120037008D06E9008E00E900D2
:10544000848060000FB99700E2C1780082FD2F00D0
:105450000F01410003F17E00800078008100E90027
:10546000050033008783D1000683D3008582D300F3
:105470000482D300F9FF3700049EBE000696BE00EA
:105480003C02BE002C03BE00E00F5200E08F5A0029
:10549000E00F5B00E08F5B008B0034000D00E0004C
:1054A000E5FF3C00880037002C60900081C6B30007
:1054B000814F50000B00320006003C000004E00069
:1054C00008003200E6C05000814F50004E003A0004
:1054D00004003700C1C6B300814F50004A003A00B3
:1054E000210037000800E00004003A005C0890004A
:1054F0008D0120000000E0000600320011000900CC
:105500000E84D8000FB99700E2C07800F1EF9F0039
:105510007D012000110009000E84D8000A00370028
:10552000110009000E04D8008D06E9000E81B900B3
:10553000020454008FB8970061417C0081FD2F0068
:105540008F80400082F07E00000478000800E000B8
:10555000020032000D00E000F1FF3C00CFC4DE008D
:10556000614DB90025003700E00F5400E08F5C006A
:1055700004003A005C0890008D0120000000E0006B
:10558000070032006171B9000800BE000003070087
:105590008FB99700E3417800F3EF9F007D01200071
:1055A0006171B9000800BE004AFA07000B0037001D
:1055B0006171B9000800BE008CF907008D06E90092
:1055C00000F1B900020454000FBA9700E4427C00D5
:1055D00084FD2F000F02420005F27E000004BE0091
:1055E000E00F5000E08F5800020032000D00E00094
:1055F000EFFF3C004FCDDE008A057800089EBE001C
:105600000A96BE0030003700E00F5400E08F5C00C7
:10561000E00F5D00E08F5D0004003A005C08900040
:105620008D0120000000E000090032006172B90025
:10563000612BB9000800BE000A01BE007D0307000F
:105640000FBA970064427800F4EF9F007D012000BC
:105650006172B900612BB9000800BE000A01BE00EA
:105660006D0307000D0037006172B900612BB900AE
:105670000800BE000A01BE00720307008D06E900A3
:1056800000F2B900040454008FBA970065427C0010
:1056900085FD2F008F82420084F27E00009EBE00B6
:1056A0000296BE003C04BE002C05BE00E00F540074
:1056B000E08F5C00E00F5D00E08F5D0002003400D1
:1056C0000D00E000E8FF3C00E80F570010003A0032
:1056D0000C1090000038A3000D003200F78F560028
:1056E00006003E0085FD2F008F824200E5C07E004F
:1056F00000C3B30080CF5000050032008D06E900E2
:1057000002C3B30081FD2F008F80400082F07E0035
:1057100078811600120E98006C00900083FD2F0017
:105720008F8141008D80410039FA07001C089000EC
:10573000DC089000810F500006003D000080500002
:10574000000E98000C1090000040A1000016980078
:105750000F0037000100E0000D003D008C109000AC
:10576000F4806000F08F500009003A007C0990003E
:10577000FC009000810051000C09900082805000D4
:10578000008050004240A90001003400000E980043
:105790004F0778004F06BE004F05BE004F04BE0005
:1057A000CF01B100000006000400FA00889FBE008F
:1057B0008A9FBE008C1F78000004780001067800E4
:1057C000F80D900078009000808555000808900042
:1057D00080855500180890008085550028089000A5
:1057E0008085550038089000808555004808900055
:1057F000808555000002220090BF9F000003230017
:10580000A0BF9F00081090000028A30015003A00D8
:105810000B00E000130034000B0578008A047800C8
:10582000E20F55000100360029002000C801900059
:1058300009017800EE805700580090000300010035
:10584000500498000000E0008C00320068089000CE
:1058500009004000600C9800090555004240A9006D
:10586000EEFF3C00780190000200E0000C003400E4
:10587000C80190008C0078005800900003000100DF
:10588000500498008080EB000000E0007C003200B3
:10589000E80890007800900000804000600C9800BC
:1058A000880C90000900E000110034000905780020
:1058B000E28F5400010036002A002000C801900049
:1058C0000A017800EC8057005800900003000100A6
:1058D000500498000000E000680032006808900062
:1058E0000A004000600C98008A845400EDFF3700E5
:1058F000180990000200E0000C003400C80190007C
:10590000E800900058009000030001005004980047
:105910008080EB000000E00059003200E8089000B1
:105920001808900000804000600C9800A80C9000BF
:105930000900E0001100340009057800E28F5400EE
:10594000010036002A002000C80190000A017800FA
:10595000EC805700580090000300010050049800AC
:105960000000E00045003200680890000A00400096
:10597000600C98008A845400EDFF370038099000CD
:105980000200E0000E003400E800900018089000CB
:1059900080804000C8019000580090000300010082
:1059A000500498008080EB000000E00034003200DA
:1059B000E80890003808900000804000600C9800D3
:1059C000C80C90000900E0001100340009057800BF
:1059D000E28F5400010036002A002000C801900028
:1059E0000A017800EC805700580090000300010085
:1059F000500498000000E000200032006808900089
:105A00000A004000600C98008A845400EDFF3700C3
:105A1000081090008000EB000028A300180032005E
:105A20000B00E000160034008B04780009057800B4
:105A3000E28F5400010036002A002000C8019000C7
:105A40000A017800EE805700580090000300010022
:105A5000500498000000E000080032006808900040
:105A60000A004000600C98008A8454004240A9005B
:105A7000EEFF3C008000EB00010037008080EB006F
:105A8000010078004F0678004F05BE004F04BE00AD
:105A90000080FA00000006000108780000000600FF
:105AA000E600400011017800050028008502610031
:105AB0006F016100820878000200320012002000AD
:105AC00011003700A0019000120020000300E00048
:105AD0000D003A00900190000300E0000A003A0037
:105AE0001000E00008003A00360037006403400070
:105AF0009608780080017800530B780090097800B0
:105B00000408780070015100110278000400E000E0
:105B1000F6FF3200130037006402400014037800DF
:105B20004F33DE00838141008308730080017800D9
:105B3000D3037800CF3BDE00140378000603430054
:105B4000068A7300130278000402420010037800F2
:105B50004F33DE008609720090017800038841000F
:105B60000201E90091017800EF8F5100EAFF360051
:105B70001000370080017800530378004F33DD00B8
:105B80001002D100040873006402400094037800FE
:105B9000CF3BDD001303D100868973001103780029
:105BA0004F33DD009401D100030A73009108D10046
:105BB0000201E80091017800FF8F5100EDFF3E00E7
:105BC000EF886100918872000200780000000600F2
:105BD0008F1FD100F80207008F87E9000000E00066
:105BE00000000600809FEB00F30207008F87E900AA
:105BF0000000E000000006002800FA00889FBE00B8
:105C00008A9FBE008C9FBE0003866B008000070049
:105C10006400E100440032006408E1004A00320000
:105C20006100E100460032006108E10049003200F5
:105C3000EC0647006000B8003D02BE003D03BE0018
:105C4000F48657006011B8003D04BE003D05BE005B
:105C50007D0320000B0037000000A0008D06E90046
:105C6000130032000402420085824A0006034B0002
:105C700087834B00000040008180480002014900FA
:105C8000838149000802520089825A000A035B009E
:105C90008B835B00F0FF3B000802420089824A00D0
:105CA0000A034B008B834B008D06E900EDFF3A00A1
:105CB0008482720086827200F707B20087827200C7
:105CC00001003200150020001E0490003E0B9000E1
:105CD00006035400E63FB0000368A300070032004B
:105CE0000000A7000500A0008301D1000281D300BD
:105CF0008180D3000080D3000603E8008301D10037
:105D00000281D3008180D3000080D3000002EB0029
:105D10000482D2001200070003F0A1000CF0A700DB
:105D200003F0A0004E003700640247006408E10061
:105D3000480032003400BE003401BE00F6FF3700D8
:105D40006108E100430032006011B8006000B80053
:105D5000F1FF370003FF270002002000FBFF3700A0
:105D60001800200057002000080453000D003D00DB
:105D70000600200097FC2F000740E1001E003400C1
:105D800084827200610260008301D1000281D3002D
:105D90008180D3000080D3000804E800F8FF3A00B7
:105DA00047002000610460000504740004046400DE
:105DB0000D00320061004000E080480060014900B1
:105DC000E081490003B8A500070032000603E8009F
:105DD0006538E10004003A008301D1000281D3005C
:105DE0008180D3000080D300F87F20000830E100DC
:105DF00003003500080378006000B8006011B800A7
:105E00004433DD00F300B20083017300000006009C
:105E1000680447000294BE000094BE00FC044700E2
:105E20008694BE008494BE0009007800AB0207008F
:105E300008007800A902070099007800814F7000DF
:105E40000B003B000800BE00840207004F00B100B9
:105E500003003700F3FF2700F2FF2F006110B900A5
:105E60004F06BE004F05BE004F04BE000080FA0082
:105E70000000060081037800B5F707000001BE00AE
:105E80006000B8000478A30013003A006220E1002B
:105E900015003E000D0039008301D1000281D300BE
:105EA0008180D3008301D1000281D3008180D3009F
:105EB0008301D1000281D3008180D3000538B00076
:105EC000C42ADD00F300B2008381720007F0A7004E
:105ED00003F0A00000000600F3FF2700F2FF2F00F0
:105EE0006110B900FBFF370003FF2700F7FF370001
:105EF0001400FA00889FBE008A9FBE008C9FBE00DF
:105F00000004BE000205BE00680047000A90BE0003
:105F10000890BE00710207000070A7000BF0A100FE
:105F2000304320009E02900080825200B0FE2F007D
:105F30000028E10011003D00B0FC2F000028E10026
:105F4000150034001E0990008E0890007E0090001D
:105F50000501B0000201D1008180D3000080D30090
:105F60008502E800FBFF3A000B00E000BCFF3B00AD
:105F700060001000E0801800B9FF3700F0FF2F002C
:105F8000F1FF27000B00E000B5FF3B0001002800F7
:105F900000002000B2FF37006000B800B0FF3700FB
:105FA0004F89DE0082017800730237000000000094
:105FB0002800FA00889FBE008A9FBE008C9FBE000A
:105FC00003866B0092FF07000028A30064003A00DC
:105FD0000128A30067003A000008A30062003A000D
:105FE0000108A30065003A001E009000BE08900062
:105FF00081064000ED3FB100F4805700EE019000B3
:10600000111AB8008E099000311BB8009E0990004B
:10601000311CB800511DB800F48557004600070038
:10602000FE0190003A0007008B85E8003E00070063
:106030008E09900040000700EE0190003400070038
:106040008B85E800380007008E09900040000700AB
:106050009E0990001B18B800890440000A8548007A
:10606000FE019000340007008B85E800380007002F
:10607000EE019000300007008E0990001B18B80058
:10608000890440000A8548000A98A30008003A00E5
:106090000402420085824A0006034B0087834B00BE
:1060A00008044C0089844C000A054D008D06E90067
:1060B00084827200850273004C3ADD008502720012
:1060C0000100320015002000443ADE001400B20046
:1060D0004538DE00CB45DD000B007000C540DE001A
:1060E000CB4DDD008B8070004549DE00CB55DD00D7
:1060F0000B017100C551DE000D03780018FF070089
:1061000003F0A1000CF0A70003F0A00054FF37003B
:106110001B18B8008502400006834800E0834B004E
:1061200060044C00070037001B18B800060340004D
:1061300087834800FAFF37001B18B8008703400028
:1061400008844800E0844C0060054D000000060013
:106150001B18B8000804400089844800FAFF370083
:106160000108A3003BFF3A005800BE005801BE00E2
:10617000E3FF37000008A30036FF3A000904780067
:10618000F9FF37000000000007F0A2000C01370003
:1061900050F707000400BE0000000600020AB90024
:1061A000001BB9000200B8008100420081004300DA
:1061B00000000600889FBE008A9FBE003004420097
:1061C000B0844A0030054B0090854B006000B10060
:1061D0000898BE000A90BE000440E10005C8E10036
:1061E00006D0E10007D8E10002003100680040005D
:1061F0001008E8004F05BE004F04BE000000060076
:10620000889FBE008A9FBE003004BE002005BE00ED
:106210000418540005985C0006185D0007985D009E
:10622000110020000440E10005C8E10006D0E100B3
:1062300007D8E100010039008000EB001088100051
:106240004F05BE004F04BE00000006001200FA0019
:10625000889FBE008A9FBE008C9FBE00E0B79F0053
:10626000F1B79F0082BF9F0093BF9F000605BE004D
:106270000404BE000000EB00D0B79F00C0B79F0031
:10628000B0B79F00A0B79F0090B79F0000067800AE
:106290005FB19700CFB09700820141003FB09700F7
:1062A0000200E00004003D00370007007E80570038
:1062B000C0FF070003003700330007007E8057004F
:1062C000CFFF0700DFB697000D00E0000C0035009F
:1062D0006FB29700FFB297000FBB97009FBB97006C
:1062E00010002000010020006011B80000027200C0
:1062F0008182720002037300838373001B00070016
:106300000C06E80001042000810F5600E0FF3A006F
:106310000D00E00004003D000802BE000A03BE00BC
:106320007E805700A3FF07005FA897000000E000F1
:1063300005003A001FB29700AFB297003FB3970035
:10634000CFB39700090007006FB09700FFB0970028
:106350000FB997009FB997004F06BE004F05BE00CA
:106360004F04BE000080FA00000006000100070094
:1063700000000600A4B79F00B5B79F00C6B79F00F6
:10638000D7B79F00000006004F09DE008281710030
:10639000B3B79F004F01DE00818040008280700013
:1063A000A1B79F008FB097004F09DE0000004000AA
:1063B0000200700090B79F007FA897004F01DE0099
:1063C000818040008280700081B79F000D0007002F
:1063D0004F3ADE000000400004007000F0AF9F0064
:1063E000080007000402420085824A0006034B00B1
:1063F00087834B00DFFF07000802BE000A03BE00D0
:10640000000006002FB29700BFB297004FB397006D
:10641000DFB3970000000600881F780018002000F6
:10642000881F780089FF07008F87E9004F047800F4
:1064300000000600801FEB0084FF07008F87E90043
:1064400000000600889FBE008A9FBE00E00F50003B
:10645000E08F5800E00F5900E08F59000C003D001C
:106460006044B8006055B8000000540081805C00B2
:1064700002015D0083815D00180020001500070007
:1064800008003D00180007000004EB00050037007D
:106490000004EB000F00070002003D00120007009F
:1064A00018002000DCFF07000800E00006003200B2
:1064B0006022B8006033B8000000520081805A00AA
:1064C00002015B0083815B004F05BE004F04BE00EC
:1064D00000000600E00F5200E08F5A00E00F5B0062
:1064E000E08F5B00000006006044B8006055B80013
:1064F0000402540085825C0006035D0087835D0012
:1065000000000600889FBE008A9FBE008C1F780096
:10651000E00F5000E08F5800E00F5900E08F590065
:106520000D003D006044B8006055B8000000540004
:1065300081805C0002015D0083815D001C00200001
:106540000820E10009A8E1000AB0E1000BB8E10071
:106550000D003D00080037000006EB00E00F520080
:10656000E08F5A00E00F5B00E08F5B0006003D000B
:106570006044B8006055B8000402540085825C0095
:1065800006035D0087835D00AAFF07000C00E000A2
:10659000060032006022B8006033B80000005200EC
:1065A00081805A0002015B0083815B004F06780006
:1065B0004F05BE004F04BE000000060000000000B2
:1065C0002800FA00889FBE008A9FBE008C9FBE00F4
:1065D00007067800878669000C003B0003047800FA
:1065E0008704780008F0A10009F0A100840F500092
:1065F000858F5800860F5900890F5C000300330017
:106600000CF0A20001003A000CF0A10000FE07000F
:106610006400E1005F003200780147006408E10097
:10662000610032006C014700748557003200BE00E3
:106630001201BE003A04BE001A05BE001E039000FF
:10664000BE0A90008503530006003D000004FD00D3
:106650008104FD000205FD008305FD008703EA00BB
:10666000050378000DF8A300040032006004140054
:10667000E0841C0060051D00E0851D006022B8005C
:106680007D0320000D38E1008006EB000B0039008F
:106690004433DD00F300B20083017300390037009A
:1066A000848272000D027800E10664008B85D100BF
:1066B0000A85D3008984D3000884D3008703E900C6
:1066C000F7FF3B0008004000898048000A014900AC
:1066D0008B81490004003B0060001000E08018003E
:1066E00060011900E08119000358A300090032007D
:1066F0008D82720084827200610260008301D10089
:106700000281D3008180D3000080D3000603E8001B
:106710001B0037000348A30017003A000600E00002
:10672000170034000603E9000D00A3000000480034
:106730008180480002014900838149000348A30089
:106740000F003A000600E000090034000603E900EB
:106750000000400081804800020149008381490017
:1067600001003A000003EB000348A300F5FF3200EC
:106770006022B800020037008482720061826600E5
:1067800077FD070003F0A1000CF0A70003F0A000C4
:10679000B3FD3700640147006408E10002003A00DD
:1067A0000DF8A300ABFD3A003200BE001201BE009E
:1067B000ABFD370000000000889FBE008A9FBE002E
:1067C0008C9FBE000404BE000605BE00809FBE0074
:1067D000829FBE002F000700040678000800BE005C
:1067E0000A01BE002B000700840678004F03BE009C
:1067F0004F02BE008D4F76007FB09700130033002C
:10680000F0FF2F008B8F6B0006003B000D0666002B
:106810000C00A7000A00370007F0A60010002000B7
:106820000A003700880F5200898F5A008A0F5B00D8
:106830008B8F5B00030039001000200001003E0038
:106840000000200007F0A7000000EA004F06BE008D
:106850004F05BE004F04BE0000000600E482400069
:106860001078A30007003200640240001178A300F2
:106870003400BE001401BE00040032000330A70043
:10688000000006003500BE001501BE000330A00068
:106890000000060005FF27000582610007003200A6
:1068A0000428E10001003200240005000600070072
:1068B00001003A004400050004080500020007003A
:1068C000F9FF3A00140005006F8261008102700038
:1068D00085027100850272000000060080007800C9
:1068E0005002BE005003BE004439DE00F700B20083
:1068F000F37F200003016100090032000218E1006B
:1069000016003A00850172008301730083817300D1
:106910000008200015003A00400020001300370056
:1069200085017200830173008381730005003A00C2
:1069300004A8BE0006A8BE00100020000B0037000F
:106940000201E9000402420085824A0006034B006E
:1069500087834B000748A300F9FF32000740A000DF
:1069600004A8BE0006A8BE002000200080009800F9
:106970009200980000000600881F78000304780049
:106980000300E00007003D0060001000E0801800F8
:1069900060011900E081190002003B0001F02D00A8
:1069A000030037000400070008F0A70003F0A00070
:1069B0004F04780000000600889FBE00008270002F
:1069C000040271000482710024003200364320006A
:1069D000C50020008383CF000A0039000541B100C3
:1069E0008283CF00070039000541B1008183CF00C9
:1069F000040039000541B1008083CF000100390057
:106A00000541B10085C353006022B8001200320076
:106A10000A003B0084827200610260008301D100A1
:106A20000281D3008180D3000080D3000603E800F8
:106A30008743E800F7FF3A000700370000004000F6
:106A40008180480002014900838149000603E90072
:106A50008743E900F9FF3A00C1FC07004F04BE007C
:106A60000000060012010000000200000200000009
:106A700000080000D80400000A0000000001000027
:106A800001020000030100000902000043000000B1
:106A90000201000000C000003209000004000000F4
:106AA00000010000020200000100000005240000B7
:106AB0000010000001040000240200000205000094
:106AC0002406000000010000052400000100000071
:106AD0000107000005810000030A00000002000019
:106AE0000904000001000000020A0000000000008C
:106AF0000007000005020000024000000000000046
:106B000007050000820200004000000000000000B5
:106B10000403000009040000340300004D000000DD
:106B20006900000063000000720000006F000000B8
:106B300063000000680000006900000070000000B1
:106B40002000000054000000650000006300000009
:106B5000680000006E0000006F0000006C00000084
:106B60006F000000670000007900000020000000B6
:106B7000490000006E000000630000002E000000CD
:106B800026030000550000004D0000004F000000EB
:106B90004700000049000000320000002000000013
:106BA0005300000065000000720000006900000052
:106BB000610000006C000000200000007000000078
:106BC0006F00000072000000740000000A03000063
:106BD00044000000340000003000000035000000D8
:106BE00044B5000088B500008CB50000C0B50000B9
:106BF000E6B50000754D00006F67000069320000C7
:106C00002D25000030320000692000007265000070
:106C100061640000792E000000250000352E000080
:106C200031660000002500003469000020000000EB
:106C3000253500002E320000660000000D0A00001D
:106C400000000000007500004D6F00006769000043
:106C50002D3200000D0A0000000D00000A000000A7
:106C60003F0D00000A0000000200FA009EC0A900CB
:106C70000080EB00702488000080EB005024880026
:106C8000AA24EF00420020008000EB00C04A200050
:106C9000E6F407002000200030258800A824EF003B
:106CA0008644A900F009200080248800F009200013
:106CB0006024880082C4A8008804A80000A02000E6
:106CC0004800DE00C02488000040EB00004F780040
:106CD000070037001E80FB00C200DD0000A020007E
:106CE000008140006000B8000089BE001E4FE8002F
:106CF0001E407800EB4F5000F6FF36009424A800A9
:106D00009624EF0094A4A9009424A90080002000F8
:106D1000502488007A69EF008069EF0081C9BF00C4
:106D20006040600081E9B70082C9BF006040600038
:106D300082E9B70050248000680060000000E00095
:106D4000F2FF3A0010C0B30095E9B70010C0B300DD
:106D500096E9B7009769EF009869EF008969EF003D
:106D60000040EB00004F7800170037001E80FB004A
:106D70008000400000972000008040008000EB0071
:106D8000010878001E80FB0080004000A0962000D3
:106D9000008040008000EB00010878009E80FB002E
:106DA000D0982000008040008040EB00014878002F
:106DB0009E80FB0000992000008040008040EB0096
:106DC000014878001E4FE8001E407800E24F500056
:106DD000E6FF360080A02000804B8800D000200015
:106DE00050258800F09920001050880080C0B30022
:106DF00000EAB70040C0B30001EAB70001CABF0013
:106E00000074A00001EAB7006269EF009A29EF0060
:106E10009C29EF009E69EF006029EF000080FA00D6
:106E2000000006000200FA00004B8000E10F500055
:106E30000B003A00A12480000004200000806000C4
:106E40000000E00006003A000080EB0050248800BB
:106E50008C04A8008C84A80020002000004B88002F
:106E600000248000700060000000E0000700320095
:106E700010248000700060000000E0000300320079
:106E80000001200000248800AA040700402480009C
:106E9000620060000000E000020032008EC0A90025
:106EA000A100370050248000610060000000E00075
:106EB0000A00320060248000610060000000E000F1
:106EC0000600320068FF07009EC0A80040002000B6
:106ED000004B8800100020005024880050248000BF
:106EE000700060000000E0000500320060248000B7
:106EF000700060000000E000010032008004070024
:106F00000124800000042000008060000000E000F8
:106F1000030032000004200000248800AD060700B2
:106F200050248000640060000000E0001400320083
:106F300060248000640060000000E0000400320073
:106F4000120020008000EB0030072000D81007005E
:106F5000400020005024880093C9BF000004E000D6
:106F60000300320093C9BF000040E90093E9B70075
:106F700093C9BF000004E00001003A00A30107002C
:106F80005124800000082000008060000000E00024
:106F900006003200612480000008200000806000AC
:106FA0000000E00001003200390407005024800096
:106FB000620060000000E0000C00320060248000ED
:106FC000620060000000E0000800320012002000B3
:106FD0008000EB00F0FF2700B51007000080EB00F9
:106FE000702488002000200050248800004B80007E
:106FF000E30F500002003E008EC0A9004A00370097
:1070000060248000680060000000E000450032005D
:107010000040EB00004F78003D0037005024800016
:10702000680060000000E0003D0032009024800015
:10703000004078008AE9B7008AC9BF000080FB00E1
:107040004400DE00004078008BE9B700800020009B
:10705000502488008AC9BF00684060000004E00036
:1070600011003A008BC9BF000081FB008080FB004B
:1070700000992000008040009040780061C06000CE
:107080000004A200E14060000099200000004100DF
:10709000E1C06000104178000204A100814071004D
:1070A00001487800100037008BC9BF000081FB0049
:1070B0008080FB00D0982000008040009040780045
:1070C00061C060000004A200E1406000D098200090
:1070D00000004100E1C06000104178000204A100FE
:1070E00081407100014878008BC9BF000004E000B6
:1070F00002003A001B040700040037000001EB0007
:10710000A198200020072000691007001E4FE8000A
:107110001E407800E34F5000C0FF360001003700EA
:10712000000000008EC0A9000080FA0000000600E8
:107130000400FA0020479800314798003E40900034
:107140000080FB00680060000000E00003003200E7
:107150008040EB002E4090009D0107003E409000D3
:107160000080FB00640060000000E00003003200CB
:1071700011C0B3002E40900095010700A14A2000E5
:107180002E4090000080FB0000004000008F400077
:107190001E007800BE409000014878000080FA0090
:1071A000000006000800FA002047980031479800C8
:1071B00022079800634798003E4090000004E000DA
:1071C000070032002E4090000080FB00800040004D
:1071D0000097200000804000100F78000600370064
:1071E0002E4090000080FB0080004000A096200010
:1071F00000804000100F78001E0078000000E000C2
:1072000002003A000000EB0037003700AE009000AB
:107210001E007800110098001E007800EE409000DB
:10722000014878001E0078001040900002C4B300AE
:10723000824060001E007800114098001E00780017
:1072400010409000804078000134A0001E007800BB
:10725000114098001E007800104090008040780097
:107260000174A0001E007800114098003E4090007C
:107270000004E0000E0032002E4090000080FB0071
:10728000AE4090008180FB0001814000019720000A
:1072900081004100910078000120A200000140001F
:1072A0000097200000004100010878000D00370021
:1072B0002E4090000080FB00AE4090008180FB00DB
:1072C00001814000A19620008100410091007800DA
:1072D0000120A20000014000A09620000000410013
:1072E000010878001E0078000080FA000000060007
:1072F0000400FA0020479800314798002E40900083
:107300000004E00017003A00404B800081C0B30049
:1073100001487800404B8000F1992000110098004E
:10732000404B8000C1C0B30011409800404B80002A
:10733000414B8000914090000174A00011409800E2
:10734000804B800041C0B30011409800804B80000A
:10735000814B8000914090000174A0001140980082
:107360002E0037002E4090000080FB0000004000FF
:10737000800078003E4090000080FB0000804000CC
:107380004300DD008000780000A02000008F400056
:107390001E00780010409000804078000124A0007A
:1073A0001E007800114098001E00780010409000E8
:1073B000804078000174A0001E0078001140980001
:1073C0002E4090000080FB0000004000800078000C
:1073D0003E4090000080FB00008040004300DD0044
:1073E000E400400000A02000008F40001E00780054
:1073F00010409000804078000124A0001E0078001A
:10740000114098001E0078001040900080407800E5
:107410000174A0001E007800114098000080FA005E
:10742000000006000200FA00004F7800A12480004E
:1074300000022000008060000000E00051003200E7
:107440001E80FB008000400000972000008040006C
:10745000100278001E80FB00800040000097200092
:1074600000804000100078001001BE0000042000E1
:10747000010020008202780003017800800178007A
:107480000100780083826200000061008000EB0050
:10749000C000DD00000020000001BE006128B8002F
:1074A0000001710081817100028ABE001E80FB0014
:1074B000800040000097200000804000100278000B
:1074C0001E80FB00800040000097200000804000EC
:1074D000100078001001BE00000420000100200010
:1074E0000000690081806900008ABE001E80FB00E8
:1074F0009E80FB0001814000019720008100410037
:10750000910078000120A2000001400000972000B7
:1075100000004100010878001E80FB008000400050
:107520000097200000804000900078001E80FB0043
:10753000000140000097200000004100100078008A
:10754000104090000044B200904098001E80FB0064
:1075500080004000009720000080400090007800EC
:107560001E80FB0000014000009720000000410049
:10757000100078001041900000C4B3000040690082
:10758000904098000080FA00000006000000FA0019
:107590009424EF008C24EF006029EF000080FA00B3
:1075A000000006000000FA00004B80000000E00030
:1075B00014003A009424EF008C24EF0020002000F7
:1075C00030258800A824EF008644A900F009200097
:1075D00080248800F00920006024880082C4A8006C
:1075E0009EC0A800010037009404A800A0248000D9
:1075F000610060000000E000FBFF3200100020008E
:10760000004B88000080FA00000006000000FA002D
:1076100095C9BF000004A2000004E000340032005D
:1076200010C0B30095E9B70096C9BF000004A200DE
:107630000004E0002E00320010C0B30096E9B7004D
:1076400077C9BF00E24F50000C003A00804B800029
:107650008040EB0001487800804B800081C4B3007B
:1076600011409800804B8000814B80009140900039
:107670000174A000114098001D00370077C9BF00B9
:10768000E14F50001A003A008C69EF00304B800047
:1076900081C0B30001487800304B8000F199200090
:1076A00011009800304B800041C0B3001140980099
:1076B000304B8000314B8000914090000174A0005D
:1076C0001140980010C0B3008CE9B700404B800017
:1076D00081C0B30001487800404B8000F199200040
:1076E00011009800404B800001C8B3001140980081
:1076F0000080FA00000006000000FA009769EF0021
:107700009869EF0077C9BF00E24F50000F003A00C0
:10771000404B800081C0B30001487800404B80009E
:10772000719A200011009800404B800081C4B30082
:1077300011409800404B8000414B800091409000E8
:107740000174A000114098001F003700A5C9BF00B8
:107750000080FB00619A2000914078008180FB004E
:10776000C808DD000100700080007800E04B800058
:10777000808F500008003100A5C9BF000080FB00C9
:10778000619A2000914078008180FB00C808DD00EC
:1077900001007000E04B880096000700804B8000DD
:1077A000719A200011009800804B800081C4B300C2
:1077B00011409800804B8000814B800091409000E8
:1077C0000174A000114098000080FA00000006003B
:1077D0000400FA00204798003147980000A02000DC
:1077E000000F78002E4090000080FB000000400059
:1077F000800078003E4090000080FB000080400048
:107800004300DD001E0F40001E007800900078004D
:1078100001F0A100010878003E4090000004E00063
:1078200007003A002E4090000080FB0080004000DE
:10783000A0962000008040001E0878000600370057
:107840002E4090000080FB00800040000097200048
:10785000008040001E0878001E007800900078002C
:1078600001E0A100010878009E00780064804000DB
:107870009000780001E0A000010878000080FA0084
:10788000000006000000FA0094A4A900D14B80007B
:1078900000082000008060000000E00027003A009F
:1078A000019820009140780000C8B30000C060003B
:1078B0000004E0000A00320020C0B30077E9B700FE
:1078C00098C9BF000004A2000004E00001003200DB
:1078D00089FF07009669EF009569EF0043003700C4
:1078E000404B800081C0B30001487800404B8000CD
:1078F000F199200011009800404B8000C1C0B300F6
:1079000011409800404B8000414B80009140900016
:107910000174A00011409800804B800041C0B3006A
:1079200011409800804B8000814B80009140900076
:107930000174A000114098002C003700F19920003C
:107940009140780000C8B30000C060000004E0006F
:107950000F00320010C0B30077E9B70097C9BF002D
:107960000004A2000004E0000100320062FF0700F2
:107970009669EF009569EF0094C9BF000004A2006A
:107980000004E0001900320020FF07001700370054
:1079900020C0B30077E9B700404B800081C0B3003E
:1079A00001487800404B8000F199200011009800B8
:1079B000404B800041C0B30011409800404B800014
:1079C000414B8000914090000174A000114098004C
:1079D0009669EF009569EF0094C9BF000004A2000A
:1079E0000004E0000100320008FF07000080FA00F8
:1079F000000006000200FA0080C0B300004F7800CB
:107A0000E04B8000E70F50000D003E00E04B80008F
:107A1000004F780076C9BF000004E00003003A0080
:107A200010C0B30076E9B7000500370076C9BF0083
:107A3000E14F500002003A0020C0B30076E9B700E1
:107A4000E14B80001E80FB0000805000E04B88006E
:107A5000804B80001E487800709A2000304C8800CF
:107A6000D04B8000610060000000E00017003A0089
:107A700009003700314C8000C04B80001041780075
:107A8000824878008100E800314C88000000E8005E
:107A9000C04B88001E4FE9001E4078000004E00043
:107AA000F4FF3A000C003700314C8000C04B8000DE
:107AB00010417800824878008100E800314C88004D
:107AC0000000E800C04B88001E4FE9001E4078000F
:107AD0000004E000F4FF3A000080FA000000060015
:107AE0000200FA00304B8000104F78009E80FB00AF
:107AF00081C9BF000080FB0022982000124178005D
:107B00000281FB004811DD0002007000808F5000F0
:107B10000800360081C9BF000080FB0021982000CA
:107B2000914078008180FB00C808DD0001007000F2
:107B3000004F780081C9BF000080FB002198200021
:107B4000914078008180FB00C808DD0001007000D2
:107B5000800078001E80FB0000805000F10F2000A4
:107B6000810060001298200012417800604161009D
:107B7000814071008141780012982000034978000B
:107B80004800DE002198200091407800E0C06000AD
:107B900000C0700082E9B7000040EB001047980079
:107BA000200037007EC9BF000080FB00F197200055
:107BB000914078008180FB00C808DD000100700062
:107BC0009E4090000181FB00719A200081004100DD
:107BD00091407800014878000000E800F10F200093
:107BE00081006000E297200012417800604161004E
:107BF0008140710081417800E297200003497800BC
:107C00004800DE00F197200091407800E0C060005D
:107C100000C070007FE9B7001E4090000040E800FF
:107C2000104798001E4090009E4F5000DDFF390025
:107C300081C9BF000080FB0021982000914078009E
:107C40008180FB00C808DD00010070000000E0003A
:107C50001E003200404B800081C0B3000148780014
:107C6000404B8000719A200011009800304B80003A
:107C70009000780000002400008060000000E00018
:107C800009003A00404B800081C4B30011409800C5
:107C9000404B8000414B8000914090000174A00057
:107CA000114098002E003700404B800081C0B30087
:107CB00011409800404B8000414B80009140900063
:107CC0000174A0001140980025003700404B80004F
:107CD00081C0B30001487800404B8000F19920003A
:107CE00011009800404B800041C0B3001140980043
:107CF000404B8000414B8000914090000174A000F7
:107D00001140980083C9BF000080FB00419820000B
:107D1000914078008180FB00C808DD000100700000
:107D20000000E0000800320083C9BF000080FB00B3
:107D300041982000914078008180FB00C808DD0058
:107D4000010070000000010080E9A90094C9BF0093
:107D50000004A2000004E000010032002BFE070036
:107D60000080FA00000006000200FA007AE9A8008C
:107D7000420020008000EB00C04A2000ABF007006A
:107D8000020320008000EB0000A02000A7F0070005
:107D90009424A8000040EB00004F78000B0037004F
:107DA0009E80FB00D0982000008040008040EB00C7
:107DB000014878009E80FB00009920000080400070
:107DC0008040EB00014878001E4FE8001E4078001C
:107DD000E24F5000F2FF3600220020008000EB004E
:107DE0003096200091F007009424A90080A0200084
:107DF000804B880000A02000304B8800304B800072
:107E0000404B8800A1C9BF0062E9B70062C9BF004A
:107E10000004E00003003A0000012000004B88004D
:107E200006003700120020002196200010002000DC
:107E30001F0D070000022000004B88000080FA00A0
:107E4000000006000000FA00F1992000914078003F
:107E500000C8B30080CF500039003A0000CCB30016
:107E60007AE9B700A2C9BF000080FB00E20F500012
:107E700009003200E30F50001D003200E10F5000F6
:107E80002D003A0020532B00C04B88002001200019
:107E9000E04B88002A003700A1C9BF000004E000C1
:107EA00011003A00A1C9BF000080FB0000004000A3
:107EB00080007800005F2B000080400010007800F8
:107EC000C04B8800C04B80000080E8001040780064
:107ED0007CE9B700C04B8000630040001040780090
:107EE0007DE9B700160037007A69EF00140037000B
:107EF000A1C9BF00E34F50000D003E00A1C9BF0063
:107F00000080FB000000400080007800205F2B0014
:107F10000080400010007800C04B8800C04B8000FB
:107F2000104078000080FB00E04B88000400370020
:107F30007A69EF00020037007A69EF000000000064
:107F40000080FA00000006000200FA00A769EF00B6
:107F5000A869EF009FC9BF007F4060000080FB0060
:107F6000E10F50000C003200E20F50000C00320014
:107F70000000E0003A003A007AE9A80088C9BF0092
:107F80000004E0002F003200A7C9BF000014A000C9
:107F9000A7E9B700320037007AE9A80030003700BF
:107FA0007AE9A800A3C9BF006F4060000004E000A8
:107FB00026003200319A20009140780000C8B300BA
:107FC00000C060000004E00008003A00A3C9BF0040
:107FD0006F4060000080FB0080004000A096200001
:107FE00000804000100F780007003700A3C9BF00D1
:107FF0006F4060000080FB00800040000097200080
:1080000000804000100F78001E007800900078007B
:1080100000002800008060000000E0000D00320039
:108020001E00780090007800004020000080600072
:108030000000E0000900320010C0B300A7E9B7005B
:1080400007003700000000000500370000000000B6
:1080500003003700000000000100370000000000AE
:10806000D14B800000082000008060000000E0008C
:1080700005003200709A2000C04B88007A09A800E1
:1080800020C0B3007CE9B7000080FA0000000600C1
:108090000000FA0050258000620060000000E0004F
:1080A00013003200304B80009040900000C8B300B5
:1080B00080CF50000D003A00804B8000904090002F
:1080C00040C8B30080CF500008003A00304B800019
:1080D000C1C0B30011409800304B8000314B80008C
:1080E000914090000174A00011409800AA24A900BA
:1080F00000082000502488000080FA0000000600DC
:108100000000FA008284A8000001200050248800AA
:1081100010C0B30089E9B7009E69EF000001EB00D1
:108120008000EB0050072000610C07000080FA007F
:10813000000006000000FA008969EF000001EB0072
:108140008000EB0040072000590C07008284A90042
:1081500000012000002488009E69EF000080FA00E2
:10816000000006000000FA00D0C2B30093E9B70097
:108170008AC9BF000080FB000020A1000000E000D1
:108180001F003A008AC9BF000080FB004200DE00E9
:10819000004078000080FB00C200DD0000A020004D
:1081A00000804000304B8800304B8000404B8800FE
:1081B000404B80000020A200404B8800304B8000E4
:1081C0009000780000C02300808060000040230001
:1081D000808F500008003A00304B80001000900063
:1081E0008200200080007800F099200088EF0700CE
:1081F0000B000700080037003600070006003700B4
:108200008AC9BF000080FB000020A100E80F5000D9
:1082100001003A004C0007000080FA000000060050
:108220000000FA007669EF009469EF009769EF00AB
:108230009869EF008C69EF007769EF00804B800050
:10824000814B8000914090000174A1001140980082
:10825000804B80000020A200804B8800804B800073
:10826000814B8000914090000174A1001140980062
:10827000804B80000020A200804B8800404B800093
:10828000414B8000914090000174A1001140980082
:108290007A69EF007C29EF008069EF0081C9BF0097
:1082A0006040600081E9B70082C9BF0060406000A3
:1082B00082E9B700800007000001EB008000EB00BE
:1082C00030002000FA0B07006EFD07000080FA0066
:1082D000000006000000FA0077C9BF00E24F50001E
:1082E00002003A00FEFD0700150037007769EF0035
:1082F0008CC9BF000004A2000004E0000F0032009F
:10830000404B800081C0B30001487800404B8000A2
:10831000F199200011009800404B8000C1C0B300CB
:1083200011409800404B8000414B800091409000EC
:108330000174A00011409800010037008C69EF0023
:108340000080FA00000006000200FA00804B800066
:10835000100078004E00DE0061406000004F7800A1
:10836000804B80000020A200804B8800004B8000E2
:10837000E80F50000D003A00A1C9BF008080FB004B
:10838000F007200000806000B0248800B024800046
:108390000000E0000300320000012000004B8800D4
:1083A0000200370040002000004B880077C9BF0062
:1083B000E14F500025003A00804B8000719A200068
:1083C000110098008BFD070076C9BF00E24F5000F6
:1083D00009003A00804B800041C0B3001140980072
:1083E000804B8000814B8000914090000174A00080
:1083F000114098002E0037001E4078000004E00075
:1084000009003A00804B800081C4B30011409800FD
:10841000804B8000814B8000914090000174A0004F
:108420001140980022003700804B800081C0B300CB
:1084300011409800804B8000814B8000914090005B
:108440000174A00011409800190037000198200025
:108450009140780000C8B30000C060000004E00054
:108460001200320083C9BF000080FB004198200049
:10847000914078008180FB00C808DD000100700099
:108480000000E0000800320083C9BF000080FB004C
:1084900041982000914078008180FB00C808DD00F1
:1084A000010070000000010080E9A9007769EF0079
:1084B0000080FA00000006000000FA009FC9BF001B
:1084C0000046B2000004E00040003A00A0C9BF002E
:1084D0000080FB00CF80DE00B200200003002000FF
:1084E000820F5000838F58003A003E000060010068
:1084F0001A0037001B00370038003700190037001A
:108500003600370006003700090037002A00370020
:108510000B00370008003700140037001D0037003B
:108520007AE9A80080002000004B88002C0037006A
:1085300044FE07002A0037000BFE07002800370022
:1085400020962000C04B88007A09A80010C0B30014
:108550007CE9B7007AE9A800210037007AFE07001D
:108560001F003700200007001D003700A3C9BF000F
:108570008080FB003096200000804000C04B8800C7
:108580007A09A80010C0B3007CE9B7007AE9A80016
:10859000130037007AE9A800A3C9BF000081FB00DF
:1085A000119A200091407800309620000000410090
:1085B000014878000A0037000001EB008000EB0062
:1085C000200020003A0B07000500370000000000E3
:1085D0000300370000000000010037000000000029
:1085E0000080FA00000006000600FA00A1C9BF00E2
:1085F000E14F50000C003A009FC9BF007F4060006F
:108600000004E00008003A007AE9A800A0C9BF0011
:10861000E34F500003003A0010C0B30088E9B700F0
:10862000010037008869EF00A1C9BF000004E00025
:10863000E6003A009FC9BF007F406000E24F500053
:10864000E2003A00A3C9BF006F4060000004E000F0
:10865000DE003200A3C9BF006F4060000080FB0055
:10866000E20F5000D9003C00014B800000022000C6
:10867000808F5000D5003A007AE9A800319A200096
:108680009140780000C8B30000C060000004E00022
:108690000F003A00A3C9BF006F4060000080FB00DC
:1086A00080004000A096200000804000100F78005D
:1086B000A3C9BF006F4060008080FB0000992000CC
:1086C0000080400010407800404798000E003700BE
:1086D000A3C9BF006F4060000080FB008000400025
:1086E0000097200000804000100F7800A3C9BF0051
:1086F0006F4060008080FB00D09820000080400028
:1087000010407800404798004E4090006140600063
:108710000004E00004003A001E0078000020A100E0
:10872000000F7800030037001E0078000020A00032
:10873000000F7800319A20009140780000C8B30003
:1087400000C060000004E00009003A00A3C9BF00B7
:108750006F4060000080FB009E0078000001400038
:10876000A0962000000041000108780008003700B2
:10877000A3C9BF006F4060000080FB009E0078002E
:10878000000140000097200000004100010878002F
:10879000A0C9BF00E34F50002A003A001E00780035
:1087A0009000780000002800008060000000E000D9
:1087B00017003200319A20009140780000C8B300C1
:1087C00000C060000004E00009003A00A3C9BF0037
:1087D0006F4060008080FB00009920000080400016
:1087E000904078000114A00001487800080037008C
:1087F000A3C9BF006F4060008080FB00D0982000BC
:1088000000804000904078000114A00001487800EA
:108810001E00780010409000804078000124A000E5
:108820001E007800114098001E0078001040900053
:10883000804078000174A0001E007800114098006C
:10884000620037001E0078000020A200000F7800B0
:108850001E00780090007800000028000080600072
:108860000000E000110032001E007800104090006F
:10887000804078000174A1001E007800114098002B
:108880001E00780010409000804078000164A00035
:108890001E00780011409800220020009E00780001
:1088A00050002000820A0700060037001E007800F2
:1088B00010409000804078000164A0001E00780005
:1088C000114098001E0078000020A200000F7800E0
:1088D0004E409000624060000004E00006003A0054
:1088E0001E007800900078000000280000806000E2
:1088F0000000E00022003200319A20009140780010
:1089000000C8B30000C060000004E00009003A00A5
:10891000A3C9BF006F4060008080FB000099200069
:1089200000804000904078000114A10001487800C8
:1089300008003700A3C9BF006F4060008080FB00C3
:10894000D098200000804000904078000114A100E1
:10895000014878001E00780010409000B2C3B300B8
:10896000824060001E007800114098002200200024
:108970009E007800500020004D0A070006003700D6
:108980001E00780010409000B2C3B3008240600027
:108990001E00780011409800A14A2000A3C9BF0022
:1089A0006F4060000080FB0000004000008040003D
:1089B000100798001E00900010407800804078005A
:1089C0000114A1001E009000014878000080FA0008
:1089D000000006000000FA00D04C8000E14C80004E
:1089E00061004000E0804800D04C8800E14C8800E5
:1089F00089C9BF000004A2000004E00008003200A2
:108A00009EC9BF000040E8009EE9B7009EC9BF00B4
:108A10000004E00002003A0000C0EB009EE9B7004D
:108A20000080FA00000006000400FA00D24C80002A
:108A3000E34C8000028FBE00D04C8000E14C8000EF
:108A40001E01BE00800F5100818F5900F7FF3A00D0
:108A50001E00BE000080FA00000006000200FA00BE
:108A6000004F7800114798001E80FB00CF80DE0089
:108A70000201200003002000820F5000838F580065
:108A80009A003E0000600100100037001700370018
:108A90001E003700250037002C0037003300370058
:108AA0003A00370041003700480037004F003700D8
:108AB000560037005D003700640037006B00370058
:108AC000720037007900370080003700DDC2A8004F
:108AD000DD02A800DD22A800DD42A800DD62A800BA
:108AE000DC02A800CD62A90088003700DDC2A90021
:108AF000DD02A800DD22A800DD42A900DD62A90098
:108B0000DC02A900CD62A90080003700DDC2A80008
:108B1000DD02A800DD22A900DD42A800DD62A80078
:108B2000DC02A900CD62A80078003700DDC2A800F1
:108B3000DD02A800DD22A800DD42A800DD62A90058
:108B4000DC02A900CD62A80070003700DDC2A900D8
:108B5000DD02A800DD22A800DD42A900DD62A90037
:108B6000DC02A800CD62A80068003700DDC2A800C2
:108B7000DD02A900DD22A800DD42A800DD62A90017
:108B8000DC02A800CD62A80060003700DDC2A800AA
:108B9000DD02A900DD22A800DD42A800DD62A800F8
:108BA000DC02A800CD62A80058003700DDC2A80092
:108BB000DD02A800DD22A800DD42A900DD62A900D7
:108BC000DC02A900CD62A90050003700DDC2A80078
:108BD000DD02A800DD22A800DD42A800DD62A800B9
:108BE000DC02A800CD62A80048003700DDC2A80062
:108BF000DD02A800DD22A800DD42A800DD62A90098
:108C0000DC02A800CD62A80040003700DDC2A80049
:108C1000DD02A800DD22A800DD42A900DD62A80077
:108C2000DC02A800CD62A80038003700DDC2A90030
:108C3000DD02A900DD22A800DD42A800DD62A80057
:108C4000DC02A800CD62A80030003700DDC2A80019
:108C5000DD02A900DD22A900DD42A800DD62A80036
:108C6000DC02A800CD62A90028003700DDC2A900FF
:108C7000DD02A800DD22A800DD42A800DD62A80018
:108C8000DC02A900CD62A80020003700DDC2A800E8
:108C9000DD02A900DD22A900DD42A800DD62A800F6
:108CA000DC02A800CD62A80018003700DDC2A800D1
:108CB000DD02A900DD22A900DD42A900DD62A800D5
:108CC000DC02A800CD62A80010003700DDC2A900B8
:108CD000DD02A900DD22A800DD42A900DD62A800B6
:108CE000DC02A900CD62A80008003700DDC2A9009F
:108CF000DD02A900DD22A900DD42A900DD62A90094
:108D0000DC02A900CD62A900000000001E40900016
:108D10000004E00002003200CC62A800010037002D
:108D2000CC62A9000080FA00000006000C00FA00E6
:108D3000213A8000F0F32F0000806000203A880084
:108D4000D1C2A900D1A2A900D5C2A800D5A2A9006C
:108D500000402D000103200094090700D1A2A800C3
:108D6000103A8000000178000210A000600420008A
:108D70007105200023742000804978008149780023
:108D8000824978000100370000000000113A80009D
:108D900000022000008060000000E000FAFF3200C6
:108DA000103A8000000178000260A10060042000F9
:108DB00071052000237420008049780081497800E3
:108DC0008249780071368000F00F2C00008060002E
:108DD00000B0A000703688004135800000FC2F00F4
:108DE00000806000E001B3004035880081368000DB
:108DF00000FC2F00008060007000B3008036880007
:108E00007136800000FC2F00008060002001B3005C
:108E1000703688005136800000FC2F000080600012
:108E20002001B300503688004134800000FC2F0040
:108E3000008060004001B30040348800213580008C
:108E400000FC2F00008060008001B3002035880006
:108E5000B1368000F00F2C008080600000302000D0
:108E600001007000B0368800103A800000017800E0
:108E70000260A0006004200071052000237420001F
:108E800080497800814978008249780000002800F4
:108E90001008880021058000F0FF28000080600095
:108EA00000E0A000200588008460A9009460A8006C
:108EB00005E1A8000421A80021088000F0FC2F0093
:108EC000008060002008880005A1A900F122A80008
:108ED00000A02600810120003409070091178000BE
:108EE00000202000008060000000E000030032004D
:108EF00010C0B300CFE9B70001003700CF69EF0021
:108F0000F0C2A900F0E2A900F102A900F122A90033
:108F1000D9E2A900E882A900E8A2A900C9C2A90073
:108F2000C9E2A900C902A900C922A900C982A900F1
:108F3000C9A2A900004020006008880000002800A5
:108F40008008880040422F00700888000003280035
:108F5000900888004105800080FF2F00008060009D
:108F60000000A000400588008500A9009500A80029
:108F70009621EF009421EF0060002000800C880013
:108F8000910C800000FE2F0000806000C000B30044
:108F9000900C880092E1A90020002800F0088800C9
:108FA000DDE2A900EC82A900ECA2A900CD02A90093
:108FB000CD22A900CD82A900CDA2A9000000000009
:108FC00000000000CDC2A800CDE2A800CE69EF00ED
:108FD000D8E2A900E802A900D9C2A900DCE2A800F1
:108FE000EC02A800E0132000101288000000280006
:108FF0000012880000532700DB030700D0E9B70008
:1090000000002300290407007C040700C6040700B1
:10901000D0C9BF000080FB00801F7800A05F2B003C
:10902000801F7800C08A20001AEC0700E4875700F0
:10903000930407003000200050198800F0FC2F0036
:109040006019880011198000F0FF21000080600085
:109050001019880025E3A90010C0B30024E3B7006D
:109060002119800000F02100010070002019880003
:1090700001198000000E2000010070000019880016
:1090800021E3A800200320001302070082C1B300DF
:1090900011C0B30000C9B3007D020700D802A900C7
:1090A000D962A900D942A900D922A900D902A900F0
:1090B000D9C2A900C962A900C862A900005822004B
:1090C000DA0407006000B800504E8800614E880046
:1090D0000040EB00404798000040EB0050479800EC
:1090E0000040EB00604798000040EB00704798009C
:1090F000D169EF000000EB00BA080700DAF60700BC
:1091000028F90700CFC9BF000004E0003E003A0084
:10911000901680006200600000F0A7000000EA00E6
:109120000000E9004F00DE00004078000080FB00F6
:10913000610060004600DD00A11780000160A10011
:1091400001007000A0178800901680006800600081
:1091500000F0A7000000EA000000E9004F00DE0078
:10916000004078000080FB00610060004700DD00E7
:10917000A11780000170A10001007000A0178800F5
:1091800011178000001020000080600000F0A70090
:109190000000EA000000E9004F00DE000040780017
:1091A0000080FB00610060004800DD00A117800026
:1091B0000180A10001007000A01788001117800035
:1091C000002020000080600000F0A7000000EA00FE
:1091D0000000E9004F00DE00004078000080FB0046
:1091E000610060004900DD00A11780000190A1002E
:1091F00001007000A017880000A026008101200057
:109200006A0807002B013700D1C9BF000080FB00AE
:10921000E10F500013003200E10F500003003C004A
:109220000000E000060032001C013700E20F500091
:1092300015003200E30F50001C0032001701370008
:10924000F4C2A900F522A8008040EB004E40900037
:1092500002FE070000402F00110020005308070005
:109260000E013700F4C2A800F4E2A9008E48900075
:109270005E409000F9FD070000402F001100200023
:109280004A08070005013700F502A900F4E2A8002A
:109290008040EB006E409000F0FD070000B82B000E
:1092A0000100200041080700FC003700F522A9005A
:1092B000F502A8008040EB007E409000E7FD07002B
:1092C00020C0B300004F980090168000620060003C
:1092D0000000E00032003A009E007800803E20004E
:1092E00000017800110009008200D8004047980072
:1092F0009E007800803E20000001780011000900E7
:109300008200D8008000FD00000F78001E01780068
:10931000B04721000090B900C388DE004F90DE0006
:1093200000805000504798001E007800B14721008F
:109330000181B9004399DE00CF80DE0001015100B8
:10934000410620000191B900820078000100500020
:10935000000F78001E017800706626000090B900AA
:10936000C288DE004F90DE00008050006047980009
:109370009E007800706626000089B9004299DE00E0
:109380004F88DE00000051006A01B9000200780039
:1093900000805000704798000040EB00004F98009C
:1093A00090168000680060000000E00032003A0083
:1093B0009E009000803E200000017800110009000E
:1093C0008200D800404798009E009000803E200018
:1093D00000017800110009008200D8008000FD0023
:1093E000100798001E019000B04721000090B900BE
:1093F000C388DE004F90DE00008050005047980088
:109400001E009000B14721000181B9004399DE00A0
:10941000CF80DE0001015100410620000191B9001A
:109420008200780001005000100798001E01900093
:10943000706626000090B900C288DE004F90DE0002
:1094400000805000604798009E00900070662600E3
:109450000089B9004299DE004F88DE00000051000B
:109460006A01B9000200780000805000704798003F
:109470000040EB00004F9800111780000010200002
:10948000008060000000E00034003A00A008800086
:1094900050079800DE009000803E20000001780018
:1094A000110009008200D80040479800DE009000BB
:1094B000803E200000017800110009008200D800E1
:1094C0008000FD00500798005E019000B047210029
:1094D0000090B900C388DE004F90DE00008050008D
:1094E000504798005E009000B14721000181B9000B
:1094F0004399DE00CF80DE000101510041062000CB
:109500000191B900820078000100500050079800D6
:109510005E019000706626000090B900C288DE00EF
:109520004F90DE000080500060479800DE00900001
:10953000706626000089B9004299DE004F88DE007F
:10954000000051006A01B90002007800008050005C
:10955000704798000040EB00004F98001117800002
:1095600000202000008060000000E0000A003A00B7
:10957000D0C0B3004047980040C0B30050479800A7
:109580000040EB006047980050C0B300704798005F
:109590000040EB00004F98000E489000E24F500052
:1095A0003D003A00504E8000614E800002002000D5
:1095B000832C240013EA07000200200003F023009C
:1095C000EBE8070098E9070050079800DE009000DC
:1095D000803E200000017800110009008200D800C0
:1095E00040479800DE009000803E20000001780097
:1095F000110009008200D8008000FD00500798008B
:109600005E019000B04721000090B900C388DE00E1
:109610004F90DE0000805000504798005E009000A0
:10962000B14721000181B9004399DE00CF80DE00FF
:1096300001015100410620000191B900820078002B
:1096400001005000500798005E01900070662600EF
:109650000090B900C288DE004F90DE00008050000C
:1096600060479800DE009000706626000089B9000F
:109670004299DE004F88DE00000051006A01B90007
:1096800002007800008050007047980010C0B300BE
:10969000004F98000100370000000000D1C9BF0052
:1096A0000040E800D1E9B700D1C9BF0063406000C5
:1096B000D1E9B70011178000002020000080600071
:1096C0000000E00003003A00CD02A800CD22A9006E
:1096D00002003700CD02A900CD22A800CEC9BF00EC
:1096E000614060000080FB00610060004C00DD0014
:1096F0006116800001C0A1000100700060168800A2
:10970000CEC9BF000080FB000000E9004F00DE0072
:10971000004078000080FB00610060004D00DD002B
:109720006116800001D0A100010070006016880061
:10973000CEC9BF000080FB000000E9004F00DE0042
:1097400000407800CEE9B700CFC9BF000004E000B8
:1097500003003200D1C9BF000004E0005C003A0001
:10976000404E8000CF80DE0050E90700020020005C
:1097700003182400DBE80700809FBE00D0602B00A8
:10978000801F7800608B200042EA0700E6875700C0
:10979000CFC9BF000004E0000300320010C0B300D6
:1097A000BBE8B7000200370000C2B300BBE8B70057
:1097B0004119800000FE2F00008060000020A00002
:1097C000401988002023A800010037000000000095
:1097D00000198000610060000000E000FBFF320023
:1097E00000188000000F78001E007800B00C880080
:1097F0001E007800C200DD000000230001007000A0
:109800002A0207009E1F780030612B00801F78001D
:10981000C08B20001FEA0700E48757004119800031
:1098200000FE2F00008060005000B3004019880047
:109830002023A8000100370000000000001980006C
:10984000610060000000E000FBFF320000188000B3
:10985000100798009E009000811F780030612B0057
:10986000801F7800108C20000AEA0700E487570068
:10987000BC000700504E8800614E8800504E8000AA
:10988000614E8000809FBE0080612B00801F7800A9
:10989000608C2000FFE90700E6875700D18D20008B
:1098A00091407800DEC8BF0080CF50000200320037
:1098B000BB020700B2E8B70071020700C08A2000AF
:1098C000FA020700E0612B00F80207000000000028
:1098D000D40507000BFE37000400FA0010079800BB
:1098E0001E009000CF80DE000001BE0000E82300D3
:1098F00001002000BDE80700000078006300500070
:10990000000F78001E007800A010880017E2A80061
:109910000080FA00000006000000FA001602A8000D
:1099200000000000B0108000610060000000E00056
:10993000FCFF3A000080FA00000006000000FA0078
:109940001622A80000000000B01080006200600035
:109950000000E000FCFF3A000080FA000000060072
:109960000000FA001642A80000000000B0108000BD
:10997000640060000000E000FCFF3A000080FA0094
:10998000000006000200FA00000F78001E007800B8
:109990009010880000000000C1108000000024002A
:1099A000008060000000E000FBFF3A00C010800073
:1099B0004F00DE00004078000080FA000000060042
:1099C0000400FA002047980000000000B01080005A
:1099D0007F0060000000E000FCFF3A001662A80073
:1099E00000000000C0108000620060000000E00085
:1099F000FCFF320080108000004F78000000000063
:109A0000B01080007F0060000000E000FCFF3A0022
:109A10002E409000614060000080FB00610060000B
:109A20004500DD00B11080000150A1000100700070
:109A3000B01088001682A80000000000B01080005E
:109A4000700060000000E000FCFF3A001E4078005B
:109A50000080FA00000006000200FA00004F7800C3
:109A600011479800ACFF07009E00FB00E00F2000AC
:109A700000806000C3FF07001E4090000000FB0054
:109A8000C0FF0700B6FF07000080FA0000000600D4
:109A90000400FA00004F7800114798002247980010
:109AA0009DFF07009E00FB00E00F2000008060008B
:109AB000B4FF07001E4090000000FB00B1FF07004C
:109AC0002E4090000000FB00AEFF0700A4FF07003F
:109AD0000080FA00000006000400FA00004F780041
:109AE000110798008CFF07001E4078000004A000BA
:109AF0000000FB00A3FF070010C0B300B0FF070089
:109B00009E0090008048780095FF07000080FA00D2
:109B1000000006000600FA00004F780011079800C8
:109B2000220798007CFF07001E4078000004A00078
:109B30000000FB0093FF07000040EB00A0FF0700C0
:109B40009E0090008048780010C0B3009CFF070082
:109B5000AE0090008048780081FF07000080FA0086
:109B6000000006000400FA008040EB0000C9B300CA
:109B7000B9FF07008E80E80063004700010178000C
:109B80008000780000C9B300E2FF07003E4090006B
:109B90000000FB004800DD00000F78002E40900020
:109BA0000000FB001E0040004580DE00000F780032
:109BB000004020009E007800808F50000700340095
:109BC0001E00EA00CF80DE0038E807000200200017
:109BD00003E02B008BE80700060037001E0078002A
:109BE000CF80DE0031E807000200200003E0230000
:109BF00084E807000080FA00000006000600FA0072
:109C000020479800314798004247980042FF0700DC
:109C10002E4090008080FB00E00F2000008060005C
:109C200058FF0700004F78001E4078000004E00055
:109C3000030032004AFF07001E407800080037008A
:109C40003E4090000080FB004EFF07004E40900019
:109C50000080FB004BFF070041FF07000040EB00C6
:109C60000080FA00000006000400FA002047980077
:109C70003147980028FF07002E4090008080FB00AD
:109C8000E00F2000008060003EFF0700004F7800DA
:109C90001E4078000004E0000300320030FF07009F
:109CA0000040EB000D0037003E4090000080FB00BC
:109CB00034FF070021FF07002E4090000004A000A1
:109CC0000080FB002FFF070010C0B3003CFF07001F
:109CD0001047980022FF07001E4090000080FA0005
:109CE000000006000800FA00881F7800204798004E
:109CF00031479800220798006347980006FF070045
:109D00002E4090008080FB00E00F2000008060006B
:109D10001CFF0700104798001E4090000004E00060
:109D2000030032000EFF07001E40900025003700A0
:109D30003E4090000080FB0012FF0700FFFE07007E
:109D40002E4090000004A0000080FB000DFF0700E3
:109D50000040EB00004F7800140037009E80FB00AD
:109D60006E4090000080FB000000E900808F5000F2
:109D7000070032001E80FB00AE009000008440000F
:109D80000040EB000EFF0700004C78000600370093
:109D90001E80FB00AE0090000084400010C0B300A5
:109DA00007FF0700004C78001E4FE8006E4090004F
:109DB0009E40780080CF5000E8FF3900E8FE0700A1
:109DC0000040EB004F0478000080FA00000006001D
:109DD0000400FA00204798002E4090000080FB000D
:109DE0004400DE00004078006A00B90000007800FE
:109DF000804078002E4090006F40600000CF40000F
:109E00001E4078000080FA00000006000200FA0000
:109E1000004F780090C3B3009E40780080CF500080
:109E200003003E0000CDB3001E404000020037009A
:109E300090CCB3001E4040000080FA0000000600F5
:109E40000200FA00000F78001E007800401288001F
:109E50000100370000000000001280006100600077
:109E60000000E000FBFF3200401280000080FA009A
:109E7000000006000200FA00DCE2A9005000200009
:109E8000EFFF07000000EB00EDFF0700004F780038
:109E9000DCE2A8001E4078000080FA000000060006
:109EA0000000FA00DCE2A90060002000E4FF0700E7
:109EB000DCE2A8000000000000000000DCE2A900D5
:109EC00010002000DEFF07000000EB00DCFF0700B1
:109ED000DCE2A8000100370000000000E5FF0700F9
:109EE0000080FB0061006000004078000004E0009A
:109EF000F9FF3A00DCE2A90060002000D0FF070073
:109F0000DCE2A8000080FA00000006000000FA0071
:109F1000DCE2A90060002000C9FF0700DCE2A80025
:109F20000000000000000000DCE2A900100020009A
:109F3000C3FF0700F00F2000C1FF0700DCE2A8000C
:109F40000100370000000000CAFF07000080FB008E
:109F500061006000004078000004E000F9FF3A0072
:109F60000080FA00000006000400FA0010079800C4
:109F7000DCE2A90030002000B1FF07001E009000C5
:109F80004880DE00AEFF07009E009000F00F20002A
:109F900000806000AAFF07000000EB00A8FF070098
:109FA000004F7800DCE2A8001E4078000080FA0034
:109FB000000006000800FA00881F780010079800CB
:109FC0002107980032079800DCE2A9003000200049
:109FD0009BFF07001E0090004880DE0098FF0700EE
:109FE0009E009000F00F20000080600094FF0700AA
:109FF0000000EB00000F7800080037001E0078001A
:10A00000AE009000008440000000EB008CFF0700D1
:10A0100000407800004C78001E0FE8003E009000E1
:10A020009E007800808F5000F4FF3500DCE2A8002D
:10A030004F0478000080FA00000006000400FA00D7
:10A04000000F78002147980095FF0700DCE2A90087
:10A05000200020007AFF07001E0078004880DE0004
:10A0600077FF0700F00F20001E00600074FF07005C
:10A070002E4090000080FB0071FF0700DCE2A8008A
:10A0800001003700000000007AFF07000080FB009D
:10A0900061006000004078000004E000F9FF3A0031
:10A0A0009AFF07000080FA00000006000400FA0092
:10A0B000100798001E0090004800DE00004F780056
:10A0C000EC02A9001E80FB005DFF07001E0090004F
:10A0D000004F78001E80FB0059FF0700EC02A8002B
:10A0E0000080FA00000006000600FA0040479800D1
:10A0F0005147980000178000000F78005E409000E4
:10A10000614060000080FB0061006000A1178000DA
:10A110000100A10001007000A01788002117800035
:10A1200000F02F00808060004E4090000080FB0017
:10A1300001007000201788000000000000000000EF
:10A1400000000000EC22A800000000000000000059
:10A150000000000000000000EC22A9000000000048
:10A1600000000000000000002117800000F02F0018
:10A17000008060002017880001178000F00F200089
:10A180000100700000178800F422A800F402A90062
:10A1900000000000000000000000000000000000BF
:10A1A000EC22A800000000000000000000000000F9
:10A1B00000000000000000000000000010178000F8
:10A1C0004700DE006140600020479800EC22A900B3
:10A1D0000000000000000000000000002E40900081
:10A1E0000004E000EEFF3A001E007800001788002F
:10A1F000F422A9000080FA00000006000000FA0026
:10A20000F00F200020178800EC22A9000117800021
:10A2100000F02F000080600000178800F002A90005
:10A22000F022A900E822A900F422A900005023008E
:10A23000C10020005D0407008040EB0080C3B30034
:10A24000A9FF07008040EB00E0C0B300A6FF0700B5
:10A250008040EB0010C0B300A3FF07008040EB007C
:10A2600020C0B300A0FF07008040EB0060C0B30037
:10A270009DFF0700250007000080FA00000006008F
:10A280000200FA008040EB0000C8B30096FF070010
:10A290000000EB00000F780006003700C08A2000A5
:10A2A0001E0040001040780011C0B3008EFF070070
:10A2B0001E0FE8001E007800EF0F5000F7FF34007B
:10A2C0008040EB0000CCB30087FF07000000EB00EC
:10A2D000000F7800080037001E017800F0004100F0
:10A2E000C08A2000008040001040780011C0B300F8
:10A2F0007DFF07001E0FE8001E007800EF0F5000E2
:10A30000F5FF34000080FA00000006000000FA00AB
:10A310000202200001022000C08A200043E707005B
:10A320000080FA00000006000000FA008040EB0008
:10A3300000C4B3006CFF070011C0B3000040EB0085
:10A3400069FF070011C0B300A0C0B30066FF07009B
:10A3500011C0B30050C1B30063FF070011C0B300C8
:10A3600010C1B30060FF070011C0B300A0C0B3006C
:10A370005DFF070011C0B30040C0B3005AFF0700E3
:10A3800011C0B3000040EB0057FF070011C0B3003D
:10A390000040EB0054FF07000080FA0000000600B8
:10A3A0000200FA000100370000000000D18D2000FB
:10A3B00091407800DEC8BF0080CF5000FAFF320025
:10A3C000DEC8BF000081FB00D18C2000810041006D
:10A3D000114F78000040E800DEE8B700DEC8BF009B
:10A3E000F04F500001003A00DE68EF001E40780098
:10A3F0000080FA00000006000200FA00004F78001A
:10A400000100370000000000111180000020200032
:10A41000008060000000E000FAFF3A001E80FB00B0
:10A42000201188000080FA00000006000600FA00F3
:10A43000200798002E0090006101B9004218DD004D
:10A44000CE10DE00810070004210DD000001BE0071
:10A4500000402200410F2000E4E507000081EB00EE
:10A460008081EB00021F4000039748001E00780027
:10A4700040118800DD68EF00DE68EF0080B02A0040
:10A48000001188002342A8008560A90041058000D2
:10A49000F0FF28000080600000C0A0004005880098
:10A4A0009560A8000080FA00000006000400FA0091
:10A4B00010079800050037001E407800CEFF070007
:10A4C0001E0090000000E800100798001E00900099
:10A4D00010407800004F78001E4078000004E00033
:10A4E000F5FF3A000080FA00000006000000FA00C4
:10A4F0009FC9BF007F406000E14F50006C003A00F0
:10A500009FC9BF0002C6B3008240600000C2B30012
:10A5100080CF500068003A00A3C9BF000004E000EB
:10A5200003003200A3C9BF00E14F500064003A00AD
:10A53000A0C9BF000080FB0001022000810F500075
:10A540001A00320001022000810F500005003C007B
:10A550000000E0000A003200E10F50000F0032005E
:10A560005800370011022000810F50003D003200DA
:10A5700021022000810F50004100320051003700BD
:10A58000408A2000C04B880080002000E04B8800FB
:10A590007A09A8007AE9A8004A003700408A20001A
:10A5A000C04B88007AE9A80046003700A5C9BF0063
:10A5B0000080FB00619A2000914078008180FB00C0
:10A5C000C808DD0001007000F10F2000810060006C
:10A5D00012982000124178006041610081407100B2
:10A5E0000141780013982000824978004800DE007D
:10A5F0002198200091407800E0C0600000C0700009
:10A6000082E9B70000882000F10F2000810060007F
:10A61000E2972000124178006041610081407100A2
:10A6200001417800E3972000824978004800DE006D
:10A63000F197200091407800E0C0600000C07000F9
:10A640007FE9B70083C9BF006040600083E9B700BD
:10A6500084C9BF006040600084E9B70080E9A800B9
:10A660001800370000882000C04B880070002000D0
:10A67000E04B880010CCB3007AE9B7001100370036
:10A68000A1C9BF000080FB00219A20009140780002
:10A690008180FB00C808DD000100700000407800E8
:10A6A0009EE8B7007AE9A800000000000500370026
:10A6B0000000000003003700000000000100370028
:10A6C000000000000080FA00000006000000FA0010
:10A6D00000B02400010020000044880011448800DC
:10A6E0008468EF008568EF0080C0B30086E8B7009B
:10A6F0009268EF0051C1B30010C0B3008CF20700A4
:10A70000D1C1B30020C0B30089F2070003C4B30075
:10A71000028420008040EB0020C0B300A1F20700BB
:10A72000D04488009C28EF009368EF000080FA0076
:10A73000000006000600FA00000F780011079800DC
:10A74000220798001E007800E50F500012003A0022
:10A75000D04480009E009000808F500006003A0098
:10A7600003C4B300028420008040EB0020C0B3008B
:10A770008CF20700D0448800E04480009E009000E6
:10A78000808F500002003A009368EF009868EF0055
:10A7900010C0B300010037000040EB000080FA0059
:10A7A000000006000400FA00000F7800214798001E
:10A7B0009268EF00D04480000000E0000600320004
:10A7C000D0448000900078000000280000806000E5
:10A7D0000000E00022003A00D04480009040780061
:10A7E0002E40900080CF500003003100D044800004
:10A7F00090407800214798009268EF000D003700E4
:10A8000092C8BF000080FB001E004000218920008C
:10A81000914078000181FB0001842000810041000B
:10A82000914078000148780092C8BF000040E800DD
:10A8300092E8B70021892000914078002E409000D6
:10A8400080CF5000EEFF390003C4B3000284200023
:10A850008040EB0020C0B30052F20700D0448800D3
:10A8600092C8BF000080FA00000006000400FA0051
:10A87000000F7800214798009EC0A90093C8BF0030
:10A880000004E00009003A009E007800A14488001E
:10A89000AE409000828920000149780010C0B300CA
:10A8A00099E8B70010C0B30093E8B7009EC0A800B5
:10A8B0000080FA00000006000600FA002007980059
:10A8C0009EC0A90093C8BF000004E000020032004F
:10A8D0009EC0A8001F0037000040EB00004F78002A
:10A8E000AE009000110798001E4FE8001E4078004F
:10A8F000E14F40000C0032001E0090001040780034
:10A900000080FB000000EA004F00DE0000407800FD
:10A910009E0090008100E800110798000004E0000C
:10A92000F1FF3A0001003700000000002E00900007
:10A93000A04488009E407800828920000149780068
:10A9400010C0B30099E8B70010C0B30093E8B70097
:10A950009EC0A8000080FA00000006000600FA0071
:10A96000200798009EC0A90093C8BF000004E00023
:10A97000020032009EC0A8001E0037000040EB001D
:10A98000004F7800AE009000110798001E4FE800BD
:10A990001E407800E14F40000C0032001E00900085
:10A9A000104078000080FB000000EA004F00DE004D
:10A9B000004078009E0090008100E8001107980098
:10A9C0000004E000F1FF3A00010037000000000041
:10A9D0002E009000A04488009E40780082892000CC
:10A9E000014978009968EF0010C0B30093E8B70000
:10A9F0009EC0A8000080FA00000006000200FA00D5
:10AA00009EC0A900E04480000000E0000800320081
:10AA1000E044800090007800000028000080600082
:10AA20000000E000020032009EC0A8006200370073
:10AA300093C8BF00E34F500001003A009368EF0055
:10AA400093C8BF000004E00002003A009EC0A800C6
:10AA50005900370093C8BF00E24F500009003A0088
:10AA60008041EB000001EB0011C0B30020C0B30037
:10AA7000CCF10700E044880030C0B30093E8B70091
:10AA80004C00370093C8BF00E14F500049003A0026
:10AA9000818920009140780000C4B30080CF50002D
:10AAA0000300360000C4B300004F780003003700F5
:10AAB0008189200091407800014F780098C8BF003C
:10AAC0001E40500098E8B70000802000B044880085
:10AAD0009E4078001147980099C8BF000004E0002C
:10AAE0001F003A000D003700B0448000A1448000F0
:10AAF0009140780001487800B04480000000E800F0
:10AB0000B0448800A04480000000E800A044880011
:10AB10001E4090000040E900104798001E40900041
:10AB20000004E000F0FF3A0010003700B04480005D
:10AB3000A14480009140780001487800B044800032
:10AB40000000E800B0448800A04480000000E80055
:10AB5000A04488001E4090000040E9001047980083
:10AB60001E4090000004E000F0FF3A0098C8BF00CB
:10AB70000004E00009003A0000C4B3009E407800E1
:10AB800080CF500003003A0020C0B30093E8B70024
:10AB90000200370030C0B30093E8B7009E41780050
:10ABA0000280200011C0B30020C0B3007DF1070077
:10ABB000E04488009EC0A8000080FA000000060063
:10ABC0000000FA00A600070088C9BF000004E000EA
:10ABD0000100320089C9BF000040FE0051248000FE
:10ABE00000022000008060000000E00002003A0047
:10ABF00010C0B30041000700D200070010C0B3002E
:10AC00000080FA00000006000000FA0088C9BF00BA
:10AC10000004E0003600320089C9BF000004E000F3
:10AC20003300320040248000620060000000E00039
:10AC3000010032008824A9007500070000042000EC
:10AC4000002488000000000001248000000420008F
:10AC5000008060000000E000FBFF320000042000E4
:10AC6000002488000000000001248000000420006F
:10AC7000008060000000E000FBFF320000042000C4
:10AC8000002488000000000001248000000420004F
:10AC9000008060000000E000FBFF32009444A80048
:10ACA000000420000024880000000000012480002F
:10ACB00000042000008060000000E000FBFF320084
:10ACC000000420000024880000000000012480000F
:10ACD00000042000008060000000E000FBFF320064
:10ACE0009444A9005700070010C0B30001003700CA
:10ACF0000040EB000080FA00000006000400FA00AB
:10AD00002047980040248000610060000000E000BF
:10AD10000B00320040248000620060000000E00070
:10AD200007003A009EC9BF00E34F50000400360000
:10AD3000202480004300DE006140600032003700C4
:10AD40002E4090000004E0001D0032008824A9007D
:10AD50008804A8002E0007000040EB00004F780098
:10AD600009003700000420000024880000000000D3
:10AD70000124800000042000008060000000E0004A
:10AD8000FBFF32001E4FE8001E407800E44F5000E9
:10AD9000F4FF36000040EB001047980020248000AC
:10ADA000680060000000E0000200320010C0B30044
:10ADB00010479800230007001E4090001200370043
:10ADC00040248000610060000000E00002003A00C2
:10ADD00000C0EB000C0037004024800062006000DF
:10ADE0000000E00002003A00E0CFB30006003700A8
:10ADF0009EC9BF00E34F500002003E00D0CFB30019
:10AE000001003700C0CFB3000080FA000000060048
:10AE10000000FA00C469EF001000FC00F10480009B
:10AE200000042000008060000000E000020032000A
:10AE300010C0B300C4E9B7009EC0A9000080FA00AA
:10AE4000000006000000FA00C4C9BF000004E000D2
:10AE5000010032009EC0A8000080FA000000060039
:10AE60000400FA001E00FC0011028000000E200009
:10AE700000806000804D880011028000000E2000DC
:10AE8000010070001002880040092000100798009F
:10AE90000000EB00000F78000E0037001E0090004D
:10AEA000900078001E00780000014000209B2000E8
:10AEB00000004100010878001E0090008000EB00B7
:10AEC000010878001E0090000080E800100798003C
:10AED0001E0FE8001E007800E50F5000EFFF36005F
:10AEE00060248000F04D88008C24EF001024800046
:10AEF000004E88008224EF00700680004800DE00CB
:10AF0000674060000080FB00104E880000012000B8
:10AF10000024880000022000502488008EC0A90070
:10AF20008284A80071068000F08F2F0000806000EE
:10AF300000A0A000700688009EC0A8000080FA0053
:10AF4000000006000400FA004009200010079800E5
:10AF50000000EB00000F78000B0037001E007800A7
:10AF600080004000209B200000804000900078007E
:10AF70001E009000010878001E0090000080E8008C
:10AF8000100798001E0FE8001E007800E50F500023
:10AF9000F2FF3600F04D800060248800004E8000F3
:10AFA00010248800104E8000004078006740600048
:10AFB0000080FB00670060004800DD007206800032
:10AFC000F18F2F0081006100010070007006880081
:10AFD00011028000F0F12F0080806000804D800021
:10AFE00001007000804D8800804D800010028800B4
:10AFF0000080FA00000006000000FA008468EF00FC
:10B0000080C0B30086E8B7008568EF0000582200D2
:10B010000100200000448800114488000080FA00EC
:10B02000000006000200FA00881F7800004B800034
:10B03000FF0F500042003600402480006200600094
:10B040000000E00040003A0093C8BF000004E000A8
:10B0500039003A0001C4B300008E2000D1FD070082
:10B06000004F78001E4078000004E00032003200FB
:10B07000009220001200200021622B00E4E3070070
:10B08000E0C8BF000080FB00ED0F5000210032003F
:10B09000ED0F500003003C00EA0F50001F0032008B
:10B0A00017003700F1032000810F50000400320028
:10B0B000C1062000810F500006003200100037004A
:10B0C00000922000A200200031622B00D0E3070094
:10B0D0001300370000922000C18A2000DAE3070045
:10B0E0000892200000922000DDE3070000004400E9
:10B0F00032002000D1622B00C5E3070008003700B2
:10B10000009220004200200001632B00C0E30700F2
:10B1100003003700000000000100370000000000BD
:10B1200000922000CEE307000040780080407800C5
:10B1300000922000CDFD070030FE0700030037001D
:10B140000000000001003700000000004F047800FC
:10B150000080FA0000000600E00800008000000007
:10B1600000000000C60900000C0000000000000004
:10B17000600900005000000000000000000A00000C
:10B18000300000000000000000080000AC000000DB
:10B1900000000000B00900001600000000000000E0
:10B1A000AC0800003400000000000000880A000025
:10B1B0001A00000002000000686A6C00747A4C00FB
:10B1C0000000010000020000040008000010000060
:10B1D000000020002B2D230030000000300A00006A
:10B1E00058000000020000006E616E00004E410039
:10B1F0004E0069006E660000494E460000000000E7
:10B2000000000000002440000000000000000000DA
:10B2100059400000000000000088C300400000000A
:10B2200000008400D79741000080E0003779C30018
:10B23000414317006E05B500B5B8930046F5F90017
:10B240003FE903004F384D00321D3000F9487700C8
:10B25000825A3C00BF737F00DD4F1500750000006F
:10B26000F4090000020000000200000030000000AD
:10B27000D20900002200000002000000303132003C
:10B2800033343500363738003941420043444500F5
:10B29000460030003132330034353600373839005B
:10B2A0006162630064656600000000000000000049
:10B2B0000600FA00000F7800110798002207980096
:10B2C0001E00780021072000810F50001700320077
:10B2D00021072000810F50000A003C00E20F5000BF
:10B2E0002C003200E20F500003003C00E10F500040
:10B2F000230032002A003700E30F50002300320001
:10B300002700370041072000810F5000190032004C
:10B3100041072000810F5000200035005107200018
:10B32000810F5000100032001D00370060178000B0
:10B330007000600000F0A7000000EA000000E900D3
:10B340004F00DE00004078000080FB0061006000DC
:10B350004400DD00611780000140A1000100700081
:10B36000601788000E003700100020001D00070045
:10B370000B003700200020001A00070008003700EB
:10B38000D2FC07001CFF07000500370057FC070030
:10B39000030037000000000001003700000000003B
:10B3A00010C0B3000080FA0000000600F03FB100BA
:10B3B0000180B10006003500EE0309000000000026
:10B3C000403FB1000180B100FBFF3D001000B00024
:10B3D000203FB0000200350000800900000000009E
:10B3E000000006000200FA00000F780000000000D4
:10B3F0000080FA0000000600FFFFFF00FFFFFF00D3
:020000040001F9
:020000040002F8
:020000040003F7
:020000040004F6
:020000040005F5
:1057F000FFFF0000FFFF0000B62300007F3E000017
:00000001FF
